:108032001269C112812E12545B1280B31254631260
:1080420080C00269C51269C112812E12545B7F5A27
:10805200C26E1253A21254E8783F79437F607EEADF
:108062001281221254637F651253A21254E8783DA2
:1080720079417F207E4E128122306E171282E412E5
:10808200813F783F794312809E783D794112809EEC
:108092001282E41269C51251660298F8C3E796FF8C
:1080A2001819E796FE0809C3E69FF71819E69EF726
:1080B200227F5B7E06904D4312496D1F800A7F66C8
:1080C2007E1474591290C21F1252397E39E4029002
:1080D200E17866E620E73418C3E6947208E6940471
:1080E2005029C318E6941F08E69404401E7869E6F6
:1080F20020E71818C3E6940E08E69401500DC31841
:10810200E6947508E694004002D322C322E67D007D
:1081120030E7011D08E62BFB18E63CFCE43DFD229E
:10812200C3EB9FF6F71819EC9EF6F7221280D340A4
:018132000C40
:10813300E47842F608F67840F608F6227864C3E657
:10814300946AF55708E6944CF5560808C3E6945824
:10815300F55B08E694AEF55A753900AC56AD57ECAD
:10816300126D57784C126DE5AC5AAD5BEC126D573E
:108173007850126DE57F2B7E867D777C18126D1CFF
:108183007850126DD9126C28126D1C7850126DD96B
:10819300126C28126D1C7850126DD9126C28126D56
:1081A3001C7F367E847D257C64126D1C7850126D95
:1081B300D9126C28126D1C784C126DD9126C2812CE
:1081C3006D1C7F3F7EA27D607C8B126D1C785012EC
:1081D3006DD9126C28126A16126A16126DF17F3F5E
:1081E3007E807D057CE60539126C287848126DE5A2
:1081F3007F2C7E937D477C7F126D1C7850126DD946
:10820300126C28126D1C7850126DD9126C28126DE5
:108213001C784C126DD9126C28126D1C7F357EB4FC
:108223007DF87CDF126D1C7850126DD9126C281208
:108233006D1C7850126DD9126C28126D1C7F3F7E15
:10824300ED7D227CCD126D1C784C126DD9126C28F9
:10825300126A1A126A167844126DE57F317E397DEF
:108263009D7CE7126D1C784C126DD9126C28126D2F
:108273001C784C126DD9126C28126D1C7844126D47
:07828300D9126A1A126D1CEA
:10828A007F2C7E377D0C7CA3126D1C784C126DD925
:10829A00126C28126D1C784C126DD9126C28126D52
:1082AA001C784C126DD9126C28126A1A126DF17F61
:1082BA003F7E807D027C9F0539126C287844126DBE
:1082CA00E57848126DD9126D8E8E428F437844122A
:1082DA006DD9126D8E8E408F4122753900AC42AD38
:1082EA0043EC126D577848126DE5AC40AD41EC1283
:1082FA006D577844126DE57F2B7E537D507C0912B1
:10830A006D1C7848126DD9126C28126D1C784812AF
:10831A006DD9126C28126D1C7844126DD9126C2812
:10832A00126D1C7F347EF27DCD7CA3126D1C7848C1
:10833A00126DD9126C28126D1C7848126DD9126C04
:10834A0028126D1C7F3F7E0A7D2E7CAE126D1C7832
:10835A0044126DD9126C28126A16126A16784C12D7
:10836A006DE57F2B7E4F7DAF7CB2126D1C78481273
:10837A006DD9126C28126D1C7848126DD9126C28AE
:10838A00126D1C7848126DD9126C28126D1C7F353B
:10839A007EB17D4B7C95126D1C7848126DD9126C9A
:1083AA0028126D1C7844126DD9126C28126D1C7F2C
:1083BA003F7E497DCD7C45126D1C7848126DD912DD
:1083CA006C28126A1A126A167850126DE5784C12E5
:1083DA006DD9126D8E8D558E568F577850126DD974
:1083EA00126D8E8D598E5A8F5B7864E557246AF622
:1083FA0008E556344CF608E5553404F608E55B24DE
:0E840A0058F608E55A34AEF608E43559F62265
:10567F001269C1125CAF1269C57F667E00904D2220
:10568F0012496D1256EF7F5A78C41256CB1256D369
:10569F0078C61256CB1256B67F6578C81256CB1203
:1056AF0056D378CA1256CB7E2DE51B1290E17E336E
:1056BF00E51A1290E17E39E5190290E18604088619
:1056CF0003023AFA7E15E51C1290E17E1BE51B12D0
:1056DF0090E17E21E51A1290E17E27E5190290E113
:1056EF007F5A7E01E53A128EB27E0B90609FE53BAA
:1056FF0093029101E6FF08E6FE08E6FD33E4500150
:10570F00F4FC75130AE4F512F511F5107539011251
:10571F006FF6A803026DE51269C1125CAFC26E7F0E
:10572F005A7E031256661256EF1298F810000810A0
:10573F00011510022080EFE53A146004153A80033A
:10574F00753A3CD26E80DFE53AB43C05753A01807C
:10575F00F2053A80EE7E031256617E0B12566612E8
:10576F0056EF1298F810000810011510022080EF64
:10577F00E53BB40205753B158002153BD26E80DF09
:10578F00E53BB41505753B0280F2053B80EE7E0BC1
:10579F001256617F5A78C41256CB1256D312581232
:1057AF001254F878C412585378C61256CB1256B604
:1057BF001258371254F878C61258537F6578C812AA
:0B57CF0056CB1256D31258121254F899
:1057DA0078C812585378CA1256CB1256B61258378E
:1057EA001254F878CA125853306E14E53B24F45018
:1057FA000B78C9E62410F618E63427F6125859121F
:10580A0069C51251660298F87E15E51C1255F5F520
:10581A001C7E1BE51B1255F5F51B7E21E51A125558
:10582A00F5F51A7E27E5191255F5F519227E2DE5AB
:10583A001B1255F5F51B7E33E51A1255F5F51A7E3E
:10584A0039E5191255F5F51922ECF608EBF622128C
:10585A0060B778C8E6FE0886073395E0FDFC126D4E
:10586A001C7FE87E037D007C00126FF6126D1C78A7
:10587A00CAE6FE0886073395E0FDFC126FCF126D6B
:10588A001C7F807E697D677CFF126FCFEC126D539F
:10589A00126D1C7F3F7E807D0D7C1D126C28126D5F
:1058AA001C7F3D7E407D007C00126D1C78BC126D11
:1058BA00D9126C28126D1C7F3E7E807D007C0012FE
:1058CA006A1A126D1C78BC126DD9126C28126D1CE2
:1058DA007F3F7E807D007C00126A16126D1C78B4B0
:1058EA00126DD9126C28126CA0783C126DE57F40BB
:1058FA007E807D007C00126D1C783C126DD9126C82
:10590A0028126E75126D1C7F3F7EA87D007C0012E6
:04591A006D1C78B8D0
:10591E00126DD9126C28126C28126D1C7F407E00FD
:10592E007D007C00126D1C783C126DD9126C281211
:10593E006E75126D1C7F3F7EC07D007C00126C2840
:10594E00126A1A126D1C78B8126DD9126C28126D6B
:10595E001C783C126DD9126A1A7854126DE5126ECB
:10596E005F7858126DE5126D1C126C28126D1C7842
:10597E00C0126DD9126C287844126DE57854126DF0
:10598E00D9126E75783C126DE5126D1C126C2812D0
:10599E006D1C78BC126DD9126C28783C126DE57FA7
:1059AE003E7EC07D007C00126D1C783C126DD912BB
:1059BE006C28126D1C7F3F7E007D007C00126A1ADF
:1059CE00126D1C783C126DD9126C28126D1C7F3F23
:1059DE007E807D007C00126A1A126D1C78B4126DE6
:1059EE00D9126C287870126DE578C4E6FE08860729
:1059FE003395E0FDFC126D1C7FE87E037D007C007C
:105A0E00126FF6126D1C78C6E6FE0886073395E017
:105A1E00FDFC126FCF126D1C7FE07E5E7DF87CFF69
:105A2E00126FCFEC126D53126D1C7F3F7E7F7DE5A2
:105A3E007CC9126D1C7870126DD9126C28126CA074
:105A4E007850126DE57F3F7EF07D007C00126D1C5C
:105A5E00783C126DD9126C28126D1C7F3F7EC07D72
:105A6E00007C00126A1A126D1C783C126DD9126CF1
:065A7E0028126D1C7F3FA1
:105A84007E807D007C00126A1A783C126DE578BC39
:105A9400126DD9126D1C7F3F7E807D007C00126ADE
:105AA40016126D1C783C126DD9126D1C78B4126DEF
:105AB400D9126C28126C287840126DE57854126D56
:105AC400D9126EAD783C126DE5126D1C126C2878FB
:105AD40074126DE57F417E107D007C00126D1C7890
:105AE400C0126DD9126C28126D1C7F407E807D001F
:105AF4007C00126D1C7844126DD9126C28126D1C36
:105B04007F417E207D007C00126A16126D1C784451
:105B1400126DD9126C28126D1C7F407E407D007C72
:105B240000126D1C7874126DD9126C28126D1C7FD2
:105B3400407EA07D007C00126A1A126A1A126A164C
:105B4400126D1C7850126DD9126C28126D1C78508D
:105B5400126DD9126C28126D1C7F3D7E2A7DAA7CA1
:105B6400AB126C28126D1C7F3F7E007D007C0012FE
:105B74006A16126D1C783C126DD9126D1C78701265
:105B84006DD9126C28126D1C7840126DD9126CA05C
:105B9400126D1C7850126DD9126C28126D1C78503D
:105BA400126DD9126C28126C28126D1C7854126D67
:105BB400D9126A16126D1C7F4A7E517DD27CCB129B
:105BC4006C28126D8E78AC126DE57F407E007D00EE
:105BD4007C00126D1C7874126DD9126C28126D1C25
:105BE4007F3F7E807D007C00126A1A126D1C78440F
:0B5BF400126DD9126A1A126D1C785055
:105BFF00126DD9126C28126D1C7850126DD9126C5F
:105C0F0028126D1C7850126DD9126C28126D1C7FE2
:105C1F003E7E2A7DAA7CAB126C28126D1C78501226
:105C2F006DD9126A16126D1C7858126DD9126CA0AC
:105C3F00126D1C7F4A7E517DD27CCB126C28126D67
:105C4F008E126D1CAF3AEF3395E0FEFDFC126D1C0A
:105C5F007F407E7E7D057C00126FF6126D1C7F608B
:105C6F007E757D587CFF126FCF126FCF78B0126D9B
:105C7F00E578AC751B64125C8D78B0751B67753950
:105C8F0000126DD9126D1C7F0A7E007D007C001200
:105C9F0070A2A81BE513F608E512F608E511F62227
:105CAF0078647BAC12570378677BB012570312608E
:105CBF00B77F007EE47D577C00126D1C78AC126DAF
:105CCF00D9126FCF126D1C7F007E537D077C00129F
:105CDF0070A2126D3B85133B7F807ECB7DA47C0031
:105CEF00126D1C78B0126DD9126FCF126D1C7F40E0
:105CFF007E7E7D057C001270A2126D3BE513F56F61
:105D0F0004F53A85126E85116D85106C7F407E7E8D
:105D1F007D057C00126D1C786C126DD9126FF61216
:105D2F006D1C7F607E0C7DA27C00126D1C78B01202
:105D3F006DD9126FCF126FE2786C126DE578AC12DD
:0F5D4F006DD9EC126D53126D1C7F347E9C7D2B31
:105D5E007C5F126C287854126DE5126E5F785012CB
:105D6E006DE5786C126DD9EC126D53126D1C7F348B
:105D7E007E9C7D2B7C5F126C28126D1C7850126DF0
:105D8E00D9126C287840126DE57F407E007D007C34
:105D9E0000126D1C7854126DD9126C28126E751289
:105DAE006D1C7F3D7EC07D007C00126D1C78BC1288
:105DBE006DD9126C28126D1C7F3E7EC07D007C005A
:105DCE00126A1A126D1C78BC126DD9126C28126CE4
:105DDE0028126D1C7F3D7E407D007C00126D1C786C
:105DEE00BC126DD9126C28126D1C7F3E7E807D0018
:105DFE007C00126A1A126D1C78BC126DD9126C28B6
:105E0E00126D1C7F3F7E807D007C00126A16126D23
:105E1E001C7854126DD9126C28126A16126D1C7FE2
:105E2E00407E807D007C00126D1C7854126DD9125C
:105E3E006C28126E75126D1C7F3D7E707D007C008D
:105E4E00126D1C78BC126DD9126C28126D1C78BCA8
:105E5E00126DD9126C28126C28126A1A126D1C78E7
:105E6E00B4126DD9126C287858126DE57854126DF3
:105E7E00D9126E75783C126DE57854126DD9126E8A
:105E8E00AD7854126DE5783C126DD9126D1C126C02
:105E9E0028126D1C78BC126DD9126C28783C126DCC
:105EAE00E57F3E7EC07D007C00126D1C783C126D3D
:105EBE00D9126C28126D1C7F3F7E007D007C001273
:0A5ECE006A1A126D1C783C126DD99F
:105ED800126C28126D1C7F3F7E807D007C00126A48
:105EE8001A126D1C78B4126DD9126C287870126D64
:105EF800E57850126DD9126D1C126C28126D1C7841
:105F0800C0126DD9126C287844126DE57854126D60
:105F1800D9126D1C126C287874126DE57840126DD8
:105F2800D9126D1C126C28783C126DE57F407E807A
:105F38007D007C00126D1C7844126DD9126C2812F9
:105F48006D1C7F417E107D007C00126A1A126D1C48
:105F58007844126DD9126C28126D1C7874126DD9A0
:105F6800126D1C7F407EA07D007C00126A16126AAA
:105F78001A126D1C783C126DD9126C28126D1C7F98
:105F88003D7E2A7DAA7CAB126C28126D1C7F3F7E59
:105F9800007D007C00126A1A126D1C7854126DD9AB
:105FA800126D1C7870126DD9126C28126D1C783C19
:105FB800126DD9126C28126C28126D1C7858126D4B
:105FC800D9126A1A126D1C7F3F7E7F7DE57CC9124B
:105FD8006C28126D1C7F4B7E187D967C80126A1A85
:105FE800126D8E126D1C7FE87E037D007C0012709E
:105FF800A2126D3B78C8A61208A61308A60608A622
:10600800077874126DD9126D1C7F3F7E807D007CED
:1060180000126A16126D1C7844126DD9126A1A128F
:106028006D1C7F3E7E2A7DAA7CAB126C28126D1CEB
:106038007840126DD9126C28126D1C783C126DD9FB
:06604800126C28126D1C11
:10604E007840126DD9126A1A126D1C7F3F7E7F7DC9
:10605E00E57CC9126D1C7870126DD9126C28126C09
:10606E0028126D1C7F487EF47D247C00126A1A1261
:10607E006D8E126D1C7FE87E037D007C001270A277
:10608E00126D3B78C4A61208A61308A60608A6072A
:10609E00223F3F4344454647484A4B4C4D4E505194
:1060AE00525354555657583F3FE4F539F5A7906073
:1060BE00CB791078B4E493F6A308D9F92232A5C2AD
:0D60CE004A4A19DC3A885CDB3BFFD6DC3B1C
:1069C100D2D58002C2D575A70490040078107F0B40
:1069D1001269ED78267F051269ED783C7F221269F4
:1069E100ED786A7F0F1269ED75A7002230D506E6B2
:1069F100F008DFFB22E0F608DFFB22DA0CD9028087
:106A01000BD906303701B35005026B899237026BFF
:106A110075D9F680F9D2368002C236126BBA303699
:106A210006C86002B237C89236DAD0D9E4B8000A93
:106A3100126C01A2369237026B5E60FBB513004007
:106A41000F126C01A23692F7A2379236A2F7923753
:106A5100C398F40424E740DF2419AD29AC28AB27FF
:106A61007A00C394084008CDCCCBCAE4CD80F4248D
:106A7100086010F9C3ED13FDEC13FCEB13FBEA13F3
:106A8100FAD9F1A236303701B340308A17E5102B1D
:106A9100F518E5113CF519E5123DF51A501A13F5F3
:106AA1001AE51913F519E51813F518E51713F51774
:106AB1000513E51370020514026B14E4C39AF5176C
:0C6AC100E5109BF518E5119CF519E51295
:106ACD009DF51A500DB237C378177F04E496F6087A
:106ADD00DFFA7A047019E513C39408F51350021503
:106AED0014E4C517C518C519F51ADAE8026BB520F7
:106AFD00E7BAE5137002151415137817C37F04E672
:106B0D0033F608DFFA80E8E51A20E7137817C37F1C
:106B1D0004E633F608DFFAE513700215141513E5D4
:106B2D00173378187F03E63400F6500E08DFF7753B
:106B3D001A800513E51370020514E51420E754704F
:106B4D0027E513604E046020851A128519118518EA
:106B5D00105326F0AC10AD11A237E51313FFE5125B
:106B6D0092E7FEA813026D3BE4F512F511F510F551
:106B7D00147513FF5326F043260580D8E5FFF51253
:106B8D00F511F510751400F513D2375326F0432681
:106B9D000980C15326F0432603E4F512F511F510D3
:106BAD00F514F513C23780AC5326F080EC79017AD9
:106BBD00018512F0E513A2F7339237751400F51322
:106BCD006002D2F785F012A813B8FF0809E512C2CA
:106BDD00E76001098C278D288EF0A2F7EF33047042
:016BED000A9D
:106BEE000AC2F705F00AD5F0011A146002D2F78531
:106BFE00F02922C88813C512C529C512C511C5288A
:106C0E00C511C510C527C51022DA03B80003026BE3
:106C1E0089D9028002D9F7026B75126BBA3037012F
:106C2E00B392377004D9E78005DADEB80003026B41
:106C3E00B5D9E2C3947E500215142513F5135002F4
:106C4E0005147815760008B81BFA78277915E6082A
:106C5E00FAE8FC78108AF0E608A427F709E5F03781
:106C6E00F7500989F00907E760FBA9F0B813E61998
:106C7E0019ECF8B82AD8026B14026BA0B8FFFA020E
:106C8E006B89D9FB026B75DAF6B800F0026BB512A0
:106C9E006DF1126BBA303701B392377007D9E3B882
:106CAE0000E280DBDAE1B8000280E1D9D5C8C398F2
:106CBE0050021514247F50020514F513781A76002D
:106CCE007A1A7B80C3E5109527E5119528E5129574
:106CDE00294016C3E5109527F510E5119528F511F5
:106CEE00E5129529F512E64BF6DA03026B14EB0367
:0A6CFE00FB30E703187600C3E51031
:106D080033F510E51133F511E51233F51240CA30A9
:106D1800E7DD80B6E53905396010D0F0D0E0C01065
:106D2800C011C012C013C0E0C0F08F138E128D11B5
:106D38008C1022E539146010D0F0D0E0D013D012B6
:106D4800D011D010C0E0C0F01539227920800C791C
:106D580010800479087D007E007F003392D55003AF
:106D6800126DCBEC33400FEF33FFEE33FEED33FD06
:106D7800EC33FCD9EE22EECCF5F0747E29A2D513C3
:106D8800FF92F7AEF022EF8EF0A2F7D2F73392D54A
:106D9800C3947F5006E4FFFEFDFC22942040047457
:106DA800FF80F304CCFEE4FFFAE5F0CC6012C3CC1C
:106DB80013CCCD13CDCE13CECF13CF0450EEDAECD7
:106DC80030D5D7C3E49FFFE49EFEE49DFDE49CFC20
:0C6DD80022E6FC08E6FD08E6FE08E6FFE7
:106DE40022ECF608EDF608EEF608EFF622CFC5130E
:106DF400CFCEC512CECDC511CDCCC510CC22E493D7
:106E0400FCA3E493FDA3E493FEA3E493FFA322C0B5
:106E1400E0126D1C126C28126E46126E02D0E0C095
:106E2400E0126D1C126E3D126C28126D1C126E0263
:106E3400126A1AD0E0D5E0E722AC48AD49AE4AAFB9
:106E44004B228C488D498E4A8F4B2274FF7809FF60
:106E5400FEFDFCE52654F048F52622126F0604A236
:106E6400E1927F1420E015906F877404126E1380F2
:106E740029126F0630E102B27F20E0EB8C4C8D4D7D
:106E84008E4E8F4F906F9B7404126E13126D1CAC58
:106E94004CAD4DAE4EAF4F126C28307F04EF648082
:106EA400FFEE33EF337001FF22126F06C0E08C4C0B
:106EB4008D4D8E4E8F4F906FBF7403126E13126DF3
:106EC4001CAC4CAD4DAE4EAF4F126C28ECC54CFC17
:106ED400EDC54DFDEEC54EFEEFC54FFF906FAF748F
:096EE40003126E13D082126D1C22
:106EED00AC4CAD4DAE4EAF4FE58230E007126CA00D
:106EFD00B27F809D126C9D8098EE33EF33246050ED
:106F0D0007D0E0D0E0026E4FEFA2E7547F927FFFF3
:106F1D00126D1C7C837DF97E227F3E126C28EE3330
:106F2D00EF3324815010126D1C126D8E126D53EFC4
:106F3D00B2E7FF126A1AEE33EF33602A2403F8C367
:106F4D0013FFEE92E7FEE82481E4501A126D1C1235
:106F5D006D8EEF04C2E0FCF582126D5BEFB2E7FFC0
:106F6D00126A1AE58203FAEE33EF33600B148FF0D9
:106F7D00A2F713FFEE92E7FEEA2283FA703AE4E9F4
:106F8D00AABCF8E0813EE6E99DBF0000803F1A3CB7
:106F9D002839666999BBE335A33DE75D25BFDB0F56
:106FAD00C93FCCDB8D41EE3649C43F91C9453DF813
:106FBD00B0C50000803F34F517C373FA2F45DDFDD2
:106FCD000AC6EF2513FFEE3512FEED3511FDEC353A
:106FDD0010FC026D3BC3EF9513FFEE9512FEED9580
:106FED0011FDEC9510FC026D3BEFF88513F0A4FF3D
:106FFD00E513C5F0CEF9A42EFEE435F0CDFA88F0F8
:10700D00E512A42EFEED35F0FDE433CC8513F0A48E
:04701D002CFCE51250
:107021008AF0A42CFCE51189F0A42CFCE51088F071
:10703100A42CFC89F0E512A42DFDEC35F0FCE51142
:1070410088F0A42DFDEC35F0FC8AF0E513A42DFDAC
:10705100EC35F0FC026D3BE4CCF8E4CDF9E4CEFA7A
:10706100E4CFFB75F020C3E51333F513E51233F5D7
:1070710012E51133F511E51033F510EF33FFEE335F
:10708100FEED33FDEC33FCEF9BEE9AED99EC98406D
:107091000CFCEF9BFFEE9AFEED99FD0513D5F0C6B2
:1070A10022C2D5EC30E705B2D5126DCBE51030E741
:1070B1000DB2D51270C5127058126DCB80031270CB
:1070C1005830D515C3E49513F513E49512F512E480
:0A70D1009511F511E49510F5102259
:1070DB00E57124885002D219123EA21242A6124226
:1070EB003C12667D1241EF12292D12310930121814
:1070FB0012711D127133127232127254305103021B
:10710B0072DE1275AF205109C251E4F552F545F507
:10711B00442275A75490040005A79005007FB4E4A2
:10712B00F0F0DFFC75A70022127A45C2517B077A7B
:10713B00FFE4FFF5A7900400127216ED244C4032C9
:10714B0075A7008D8205A71271DC7583058D82E012
:10715B002410401CF005A7E02CF0500505A7E00417
:10716B00F0BA000CBB0009D251EF24DC50027F2394
:10717B00DFC6EA600512718F8006EB60031271C7E0
:10718B0075A7002230E0047553082230E1047553D3
:10719B00182230E2047553282230E3047553382249
:1071AB0030E4047553482230E5047553582230E619
:1071BB00047553682230E7037553782230E0047569
:1071CB0053882230E1047553982230E2037553AA99
:1071DB0022ED54F0C423239071E6735302FE225325
:1071EB0002FD225302FB225302F7225302EF2253DA
:1071FB0002DF225302BF2253027F225303FE22538C
:0B720B0003FD225303FB225303FB2270
:10721600127958127841E4F5F7C2B2C2B2ADF7F569
:10722600F7C2B2C2B2ACF7D2B2C220229005007841
:10723600B4E06015FD54F0C4CD7C00540FFE1583F8
:10724600E0FF123C30EFF005830582D8E422758317
:107256000478FF088882E060FAF5D38812E51224E4
:107266004C50012285D3D288D4881279FF0512E5C5
:107276001260F00908E875F0B484A8F08882E0602E
:10728600ECF5D3B9000280D5B9230050D0C395D20E
:1072960092D15002F40409FEE4FFFCAD01123C3D1C
:1072A6007401FA25D475F0B484A8F0AC06AB0712C5
:1072B6003B24EB30E7010CE5D22C30D1029C9C88B4
:1072C60082F00AEAB501DCE512244C50012285D38E
:1072D600D28512D4A812809390040012739D8C0656
:1072E6008B0512739DE4FFF512F5118C148B13C3F5
:1072F600ED9BF9EE9CFA4012E51199E5129A500AB7
:107306008C148B138A1289118F528F82E0F9C3ED88
:0673160099FDEE9400FE5B
:10731C00E582245A5002244C75F0B48485F082E046
:10732C00FA2DFDEE3400FEEB9AFBEC9400FCE92BFD
:10733C00FBEC3400FC0FBFB4B0E55224D340022464
:10734C00B4F552C3E51333FBE51433FCE511FE2B06
:10735C00FBE512FF3CFC123C92E9F89073AF93F5FD
:10736C0011FDEBF513FFECF514FE7C00123C308F95
:10737C0044E89074AF93FAAB13AC14123B5BAF03BD
:10738C00AE04AD117C00123C30EF7002F552F545A5
:10739C00227C007B007F5AE02BFBEC3400FC058246
:1073AC00DFF522B4B4B4B4B4B4B4B4B4B4B4B4B4B7
:1073BC00B4B4B4B4B4B3B3B3B3B3B3B3B3B3B3B38C
:1073CC00B3B3B2B2B2B2B2B2B2B2B2B1B1B1B1B194
:1073DC00B1B1B0B0B0B0B0B0B0AFAFAFAFAFAEAEA8
:1073EC00AEAEAEAEADADADADADACACACACACABABC6
:1073FC00ABABAAAAAAAAA9A9A9A9A9A8A8A8A8A7EF
:10740C00A7A7A7A6A6A6A5A5A5A5A4A4A4A4A3A31F
:10741C00A3A2A2A2A2A1A1A1A0A0A0A09F9F9F9E57
:10742C009E9E9D9D9D9D9C9C9C9B9B9B9A9A9A9994
:10743C0099999998989897979796969695959594D3
:10744C009494939393929292919191919090908F16
:10745C008F8F8E8E8E8D8D8D8C8C8C8B8B8B8A8A58
:10746C008A8989898888888787878686868585859D
:10747C008484848383838282828181818080807FE3
:10748C007F7F7E7E7E7E7D7D7D7C7C7C7B7B7B7A24
:10749C007A7A797979787878777777767676757568
:1074AC00757474000203050608090B0C0E101113F9
:1074BC00141617191A1C1D1F2122242527282A2BC4
:1074CC002D2E303133343637393A3C3D3F40424330
:1074DC00454648494B4C4E4F505253555658595AA5
:1074EC005C5D5F606163646667686A6B6C6E6F702D
:1074FC007273747677787A7B7C7E7F8081838485C7
:10750C008688898A8B8D8E8F909192949596979878
:10751C00999B9C9D9E9FA0A1A2A4A5A6A7A8A9AA41
:10752C00ABACADAEAFB0B1B2B3B4B5B6B7B8B9BA27
:10753C00BBBCBDBEBFC0C0C1C2C3C4C5C6C7C7C823
:10754C00C9CACBCCCCCDCECFD0D0D1D2D3D4D4D53C
:10755C00D6D7D7D8D9DADADBDCDCDDDEDEDFE0E06B
:10756C00E1E2E2E3E4E4E5E5E6E7E7E8E8E9EAEAB4
:10757C00EBEBECECEDEEEEEFEFF0F0F1F1F2F2F311
:10758C00F3F4F4F4F5F5F6F6F7F7F8F8F8F9F9FA88
:10759C00FAFAFBFBFBFCFCFDFDFDFEFEFEFEFFFF15
:1075AC00FFFFFFC251E4F544F814FB900400A9005E
:1075BC007C0FC2D11276CAE82405F8B8B4F08B134C
:1075CC00E5122403FA244C5001FABBFF0122751179
:1075DC002C8A191277018F16206F12AA1975112394
:1075EC001277018F15751600306FE280117511231B
:1075FC001276A9751500306F05E82F13F515751166
:10760C00121276A9751400306F05E82F13F514EAE1
:08761C002404F552244C500235
:10762400F552E4F51AF51BF51CE516600AFB7A0021
:10763400AF137EFF12766FE515600AFB7A4FAF1326
:107644007EFF12766FE516600DFB7A00E514600686
:10765400FF7ECF12766FAE1CAF1B7C00AD1A123CBE
:10766400308F45EF2513F544D25122EFF5F0A4FCF9
:10767400ADF0EBF5F0A49CFCE5F09DFDEB8AF0A4E5
:10768400FAABF0EF8EF0A49AF8E5F09BF9E833F842
:10769400E933F97B00123CD6051AE51B2BF51BE4F4
:1076A400351CF51C22EA2511F9244C5001F9C2D1EC
:1076B4001276C8306F428F00C3EA9511F950032443
:1076C400B4F9D2D17C09E4FDFEFF8982E060062F83
:1076D400FFE43EFE0D09B9B4027900DCEDED20D1E2
:1076E40018F51E24FE926F500F123C3DEFB50300B7
:1076F4005006851E1FFB881222F51D80E61276A90E
:10770400206F4374021277A01276A9206F38740494
:107714001277A81276A9206F2D74061277A012761C
:0C772400A9206F2274081277A81276A921
:10773000206F17740A1277A01276A9206F0C740CB0
:107740001277A81276A9206F0122C3E89F605088A3
:10775000148F158A1640081ABAFF0A7AB380060AEF
:10776000BAB4027A001276A9306F34C3E89FF96088
:107770002EC3E5149515FB6930E7D4E930E703F42F
:1077800004F9EB30E702F404C3995002AA16E51499
:107790002515C82F28FFE4FC33FE7D04123C30225F
:1077A0002AFA244C5001FA22C3CA9AFA500324B48C
:0277B000FA22BB
:1077B200C2B2129A17D2B275F83022C2B2F5F7C22B
:1077C200B2C2B2D2B222D220D21474061277BD74DF
:1077D200C71277BD1206451277E5123872801F7400
:1077E200FF8001E4F5BCF5BDF5BEF5BF22120645EA
:1077F20085BF6C85BE6B756A0012785EC22FD2207F
:10780200C2B275F705C2B2C2B2C2B2C2B275F70550
:10781200C2B2C2B2C2B2C2B2E5F7540170EFD2B282
:10782200C22022D220C2B2F5F7C2B2C2B2856CF730
:10783200C2B2C2B2856BF7C2B2C2B2856AF722D2B5
:1078420020C2B275F703C2B2C2B2856FF7C2B2C22A
:10785200B2856EF7C2B2C2B2856DF722E56B7017C0
:10786200E56A7013D22012780074061277BD74D8BC
:10787200127825D2B2D22FC22022127800D22074DE
:10788200061277BD74021278258FF7C2B2C2B2D245
:10789200B2C22022852E72E55F030354C0F8E55E72
:1078A200543F28F57C30550122202F0612785E3095
:1078B2002F25D220C2B275F705C2B2C2B2C2B2C27D
:1078C200B275F705C2B2C2B2C2B2C2B2E5F7540192
:1078D200D2B2C220600122C22F127B7178BFE6238E
:0878E200C454E0F8E575F94813
:1078EA00F5751278F2897522127800D22074061280
:1078FA0077BD7402127825787086F708B880FAD2B4
:10790A00B2C2207410256A54F0F56AE4356BF56B3F
:10791A00E4356C540FF56C22E56A240180EBD380C0
:10792A00EAE54B75F010A4256A54F0F56AE5F08093
:10793A00DBE56A24F054F0F56AE56B34FFF56BE594
:10794A006C34FF80CEE56A24FF80ECC380EBE56DE2
:10795A0024F054F0F56DE56E34FFF56EE56F34FFF3
:10796A00540FF56F22D3E4356EF56EE4356F80F06F
:10797A001279D8127A04C254C255E57F7002D255E0
:10798A00147002D254E54A30E00122B40620205491
:10799A000F12793B127ABC127B50127B88027C044C
:1079AA001260DE7E04129A13754A01D256222055BD
:1079BA000F12790D127B2F127B71127A95027BD7E7
:1079CA001260DE7E04129A13754A05D25722740396
:1079DA001278257870E4F5F7C2B2C2B2A6F708B8F1
:1079EA0080F3D2B2C220227403127825E4F5F7C2DA
:1079FA00B2C2B2E5F7D2B2C22022E575F8541F30FE
:107A0A00E40244E0F575E803C4540778BFF679C286
:017A1A00C3A8
:107A1B00E796E6F750031263BC85722EA277922687
:107A2B00E57C543F30E50244C0F55EE57C54C02351
:107A3B0023F55FE57F1414F55122856C6F856B6E12
:107A4B00856A6D22856F6C856E6B856D6A22E4FE8F
:107A5B00FF740775A704F5838E8274FFF0DFFD7545
:107A6B00A7002274067E007FB0127A5EE4F55AF509
:107A7B005B2275A704758306E55A600A75F00A84C4
:107A8B00E5F07002740AC4F58222307720E55A249F
:107A9B00024002055A127A7DE55AF0E573F0E5745F
:107AAB00F0E575F0E576F0E577F0E578F075A70091
:107ABB00223077F9127A7D7F1074FFF0DFFDE55AE3
:107ACB0024F55003127AE7155AE55AB4FF02055A0A
:107ADB00C3E55A955B50D6755B0080D1127A457F12
:107AEB000A056D056D127841E4F5F7C2B2C2B2E535
:107AFB00F7D2B2C22030E704DF028005127958803A
:107B0B00E0056D127841127A7DE55A24F6F07F0676
:107B1B00E4F5F7C2B2C2B2E5F7F0DFF4D2B2C2209D
:107B2B0075A70022053FE53FB43C17753F00053EA6
:0A7B3B00E53EB43C0D753E00053D2B
:107B4500E53DB41803753D0002337B153FE53FB4B1
:107B5500FF17753F3B153EE53EB4FF0D753E3B15E2
:107B65003DE53DB4FF03753D1702337B0542E54214
:107B7500B43C0F7542000541E541B43C0575410033
:107B85000540221542E542B4FF0F75423B1541E51C
:107B950041B4FF0575413B154022E54075F03CA415
:107BA5002541FBE435F0FC7A3C123B24EB2542FBF6
:107BB500E43CFC22E53D75F03CA4253EFBE435F0B4
:107BC500FC7A3C123B24EB253FFBE43CFC22207471
:107BD5000122C3E5709557FF24FD5021EF24EB40AA
:107BE5000A78B906B6001618068012EF2402400D71
:107BF500EF2414500878B706B600021806802BC388
:107C0500E5709557FF24FD5021EF24EB400A78B726
:107C150016B6FF1618168012EF2402400DEF241435
:0E7C2500500878B916B6FF021816857057225F
:109A09007E0480067E0280027E017F0080047F0141
:109A19007E00EF4E6012E4FD0D1D0DEDC394AD40C7
:099A2900F7EF1F70ED1E80EA2228
:109A7700F5D8D2DCE5F520E7FBE5DA540FFEAFD9E0
:049A870075D800226C
:109728007F767E0690979112493C7404129A777C52
:10973800007D52123C30EFF875F00A84C0F07F7655
:109748007E231290E17E29742E1291017E2ED0E0A4
:109758001290E17E3574561291017F6B7E119097BD
:1097680096129053E824E04001220423F824E7509D
:10977800027818129781D8FB227F6CE82411FE79B1
:109788000512997C0E0FD9F9224143435500071D54
:10979800FFFFFFE080000020C0000038E000000864
:0C97A800F0000038F8000020FFFFFFE098
:10989D0075F0FF800875F02D800375F005E41098C4
:1098AD000A850707D5E0F7D5F0F422E5996238224D
:1098BD001298A230E6022409540F75F00AA4F5158A
:1098CD001298A230E6022409540F2515221298A2EF
:1098DD00540F221298EAC4FA1298EA2A221298A278
:0B98ED0020E603540F22540724092238
:1094CA00E61294D118E608FAC41294D7EA540F4463
:1094DA0030F924C6E9501624078012753800800D29
:1094EA0075F00A84C0F01294F5D0E0443020530B92
:1094FA0075F000850707D5F0FA801BC0E030981494
:10950A00C298E599B4130D10020A3098FAC298E588
:10951A0099B411F3D0E03099FDC299F599623822D5
:10952A00E5381294D180081294F7E5381294F7744A
:10953A000D1294F7740A80B574401294F780AE74D1
:10954A002C80AA742E80A6741180A27413809E1295
:10955A007B9F12954274491294E578041294CA804A
:01956A00BF41
:109A9D0085A08485A0835383FE438380F075840065
:019AAD002296
:10956B0074A2129A9D74A1129A9D74C0129A9D7442
:10957B0025129A9D1295ED75C70375C6FC75B90139
:10958B001295BE24EA50027E16EE9095D69325BC1A
:10959B00FE24E6501A24E840167481129A9DEE12AE
:1095AB009A9D1295FA742F129A9D74AF029A9D7E12
:1095BB002680E67408129A77EE75F020A4FEEF541D
:1095CB00F80303032E2492C313FE22F7F7F8F8F9DE
:1095DB00FAFBFCFDFEFF000000000101020202038A
:1095EB000303A8BCA9BDAABEABBFACC7ADC622883E
:0C95FB00BC89BD8ABE8BBF8CC78DC62208
:1098F800D21AC006C007C0E075A7019000007EB765
:1099080075A700EE129A9D7410129A9D7404129A0B
:109918009D85A08485A08343838175A7517F80E0BE
:10992800F0DFFC1EBEAFD9E4F5A7F584D0E0D00780
:05993800D006C21A2256
:109A8B0075A711900000E4C583F0C58330E2F8F5AB
:029A9B00A72200
:10997C00EF20E723EE20E71F20E61C05A7C45403C5
:10998C00F583EE5408C42FF582EE5407240983F5B1
:10999C00F0E045F0F005A7228040201008040201F9
:1099AC00EF20E723EE20E71F20E61C05A7C4540395
:1099BC00F583EE5408C42FF582EE5407240983F581
:1099CC00F0E055F0F005A7227FBFDFEFF7FBFDFEBF
:10904F00C2D18002D2D1C0A7C082C083C007C006E0
:10905F00C0E030D10975A704E493FDE493FAEEFB69
:10906F0075A704EBFEEAFC7901D9067908E493F5BC
:10907F00D4E5D423F5D420E0161299AC0EDCEA0F18
:10908F00DDE1D0E0D006D007D083D082D0A7221266
:10909F00997C80E89045C77A04C0E075F005A42557
:1090AF0082F582E5F03583F583D0E07D0580917AF6
:1090BF000580027A04547FC0E0C083C082C394202D
:1090CF005001E49045771290A8803D9046C67A05EE
:1090DF00800590477C7A06C0E075F007A42582F5DD
:1090EF0082E5F03583F583D0E07D0702904F7A0556
:1090FF0080027A06547FC0E0C083C082C3942050A0
:10910F0001E490470C1290E6D082D083D0E02290F9
:10911F0044F5C0E075F00AA42582F582E5F03583A9
:0B912F00F583D0E07D0A7A0702904F24
:108E4700F5D2C2D58036F5D2D2D58030F5D224F608
:108E570050090E0E24A650030E0E0EE5D2F5D2755C
:108E6700F0648485F0D3C2D57009D2D574201291ED
:108E77000180031290E1CE2406CEE5D375F00A8473
:108E870085F0D3700A30D507742012910180031240
:108E970090E1CE2406CEE5D31290E1E5D222F5D2B9
:108EA70075F0648485F0D3C2D58022F5D2C2D5800F
:108EB70025F5D2D2D5801FF5D275F0648485F0D31D
:108EC700C2D57009D2D5742012910180031290DAAD
:108ED700CE2405CEE5D375F00A8485F0D3700A3029
:108EE700D507742012910180031290DACE2405CEA3
:108EF700E5D31290DAE5D222F5D2C2D58025F5D294
:108F0700D2D5801FF5D275F0648485F0D3C2D570B1
:108F170009D2D574201290C280031290A3CE2404E4
:108F2700CEE5D375F00A8485F0D3700A30D507747F
:108F3700201290C280031290A3CE2404CEE5D31250
:058F470090A3E5D22219
:10492E007405FEF51EE4FFF51DF51F206E3175A70B
:10493E0000E493700122A3B40204051D8003B401A8
:10494E000A051FEF2409FFAE1E80E61291017D06B7
:10495E00B440027D03B421027D02EE2DFE80D2759D
:10496E00A700E493700122A3B40204051D8003B4D2
:10497E00010F051FEF2407FFAE1E80E61290BE80CA
:10498E0008B45B0050F61290C20EB4210280D30E12
:10499E00B4400280CDB42C0280C80E0EB45F0280EB
:1049AE00C1B45B0040BC0E0E80B8E608129101EE59
:1049BE002406FED513F422E6081290C2EE2404FE5D
:1049CE00D519F4227F347E2F9049EAE53F20E00985
:1049DE009049EE2074039049F202493C20202000B9
:1049EE0056414C004241440075F019D5E0FDD5F01A
:1049FE00FA129542744F1294E5744B029531124A95
:104A0E0043C29812989DC5F06022C5F0B440F412CE
:104A1E0098A2B440031298A2B44F181298A2B44BA5
:104A2E00121298A21298A21298A2C32212989DC591
:104A3E00F070D7D322120631E5BC6402700975F00E
:104A4E0008D5E0FDD5F0FA227F0375F019D5E0FD0B
:104A5E00D5F0FA12954274571294E574501294F7E9
:0A4A6E0074811294F7E5631294F7C7
:104A7800E5621294F778D4E61294F708B8DCF87473
:104A88005F1294F71294F71294F774581294F7740B
:104A9800431294F7E41294F71294F77864E61294A8
:104AA800F708B869F8E6129531124A0C400122DF7E
:104AB80002800775F000809BD250D322124A43C26D
:104AC80050C2982002F412989DC5F060EBC5F0B46E
:104AD80040F11298A2B440031298A2B457DCF538FA
:104AE8001298A2B450D41298A21298A2F563129800
:104AF800A2F56278D41298A2F924A0500353015F5A
:104B0800E924E04002795FA60108B8DCE8780712DA
:104B180098A2D8FB78641298A2F608B86AF8129896
:104B2800A2E53870951298A21298A2C322904B4A17
:104B38007F207E0012496D1298F8029A11904B5B03
:104B480080EE205452414E534D4954204552524F05
:104B580052200040574159504F494E54204558491A
:104B6800535453400012423C129A8B1261E8029847
:104B7800F8D227C26B75480A121E02121E1D753420
:104B880000124B6DC26A1225BB106A051201A5807E
:104B9800ED124FDA125116E964FF7003124D6312D9
:104BA8005166904CB3124D741201A5206D05206F0B
:104BB8004480CB904CBD124D74206D06206FE302EB
:104BC8004C71120EFF904CC9124D74206D05206F68
:104BD800E2804BC015120F38124D93D01510000605
:104BE8001001DF1002BC120F4A124E04100006100A
:104BF80001E1100289120EFF306E11904CEF124D38
:074C080074206D18206FDF1E
:104C0F00C26E024C97904CF8124D74206D07206FB6
:104C1F00CED26E80738084125048E516700B124D01
:104C2F004F7E08129A13024B86124D4912525C1294
:104C3F0050974009124C51753500024B86124B4567
:104C4F0080F5D26B125142125019E51775F010848E
:104C5F00240AF54824E8500375480A121E2985587E
:104C6F00592212525C1250974014D26B1251427556
:104C7F001607855917121E88753500024B86E96590
:104C8F001560E7124B4580F0D26B12500275B901D7
:104C9F00E5BCB2E7F5BC12387280D4574159504F7A
:104CAF00494E5400202045584954202021002120EE
:104CBF004540444049405420210020204E4045406B
:104CCF00572020004052454345495645400021207A
:104CDF00534045404E404420210046524545400038
:104CEF002044454C455445200040524553544F52A3
:104CFF00454000454E54455220004C41542F4C4FD7
:104D0F004E00574753213834002040554054404DF2
:104D1F00402000554054404D00535749535347448A
:104D2F00004143542C504F532F4845494748540096
:104D3F00414C5400535549405800124D631251666F
:104D4F007F197E12904CE912496D7E23E516128F62
:104D5F000B0298F87862E4124D6D78D4745F7F0877
:104D6F00F608DFFC227F197E1012496D1298F8C2E7
:104D7F006DC26F10000810010810020780F5D26D88
:104D8F0022D26F22C2517F197E10904CD312496DDF
:104D9F00125048E5167008124D4F129A098050753F
:104DAF00A6FF124E361231477F207E0B12496D122D
:104DBF0098F83051031249FFC29820003220012F7A
:104DCF0020022C3098F4124AC74015D25112509736
:104DDF004018124C51125166120F381298F880A6D3
:104DEF00105003124B35C25180B5124B4580B01293
:104DFF004E360298F87F197E10904CDD12496D12D5
:104E0F004E361231477F207E0B12496D1298F820D3
:024E1F0000DDB4
:104E21002001DA10020280F5124A564003D2022212
:104E3100124B3580CE7F207E00781074201290C2F4
:104E4100CE2404FED8F5227E00780B742012910145
:104E5100CE2406FED8F522D220753200127A597579
:104E6100A70490070075150012500275B901E5BC41
:104E710020E705E515F0800C04600975BCFF75B9E4
:104E81000575B9020515E515242050DCE58224FEDF
:104E91004003024F2FA882187F0075A70075830772
:104EA1008882E0FE75F004A4124FADA9BCAABDAB87
:104EB100BEACBF1582E0FD75F004A4124FADC3E98D
:104EC10095BC404C7052EA95BD4045704BEB95BE88
:104ED100403E7044EC95BF4037703DEE75F004A440
:104EE10004124FADA9BCAABDABBEACBFED75F004B9
:104EF100A404124FADC3E995BC4015701BEA95BDE2
:104F0100400E7014EB95BE4007700DEC95BF500834
:104F1100EEF00582EDF01582E5826009C3EF95821E
:104F21005003024EA30FC3E89F4003024E9B75A797
:104F31000490070075C70375C6A8E0F5BCE0F5BD90
:014F4100E08F
:104F4200F5BEE0F5BF75B90575B90205C6E582245F
:104F5200204006E5C6242050E00875C70375C680C8
:104F620075B901E5BC124F97F5BCE5BD124F97F537
:104F7200BDE5BE124F97F5BEE5BF124F97F5BF755F
:104F8200B90205C6E5C6245850D6E5320470FB7551
:104F9200A700C22022B4FF0122F975A704900700DE
:104FA200E582686005E06970F7E922F5C685F0C719
:104FB20075B901E5BC645F700375BC27E5BD645F2C
:104FC200700375BD27E5BE645F700375BE27E5BF3C
:104FD200645F700375BF272275C703E54875F00447
:104FE200A42480F5C6E55975F00484A8F00825C606
:104FF200F5C675B901A9BCAABDABBEACBF86152268
:10500200E515242050037515DFE51575F004A45449
:10501200FCF5C685F0C722E51724204028E5177560
:10502200F00484A8F00824A8F5C675C70375B90171
:10503200A9BCAABDABBEACBFA61589BC8ABD8BBE3E
:105042008CBF12387222E4F516F51579FF12500260
:1050520075B901E5BCB4FF040516A9150515E515DA
:10506200242050E9891579FF75C70375C6A875B95B
:085072000109E5BC04601B0903
:10507A00E5BD04601509E5BE04600F09E5BF0460DB
:10508A000905C6E5C6242050DD098917227900E9F9
:10509A0075F004A454FCF5C685F0C775B901E5BCE2
:1050AA0020E73078D466702B08E5BD66702508E5E0
:1050BA00BE66701F08E5BF66701905C675B9010896
:1050CA00E5BC66700E08E5BD66700808E5BE667048
:1050DA0002D32209E9242050B6C3221251051250E4
:1050EA00EDA8017F08E0F608DFFB221251051250F5
:1050FA00FDA8017F08E6F008DFFB2278D479627503
:10510A00A704758307EBC454F0F582221250027883
:10511A00D4125130E5BCF9C26E20E702D26E1251A8
:10512A0030786212513075B901A6BC08A6BD08A62E
:10513A00BE08A6BF0805C622D22012500278D41291
:10514A005154125154786212515486BC0886BD08D3
:10515A0086BE0886BF0812387205C622129A8B7F4D
:10516A00007E09904CAA12493C7F0A7E12E515047A
:10517A00128E537F14128B6C120EFF7E097F2775D5
:07518A00130878D41249B8A4
:105191007F3D7E01904D1112496D20311B3030034E
:1051A10012567F78661253D01251BE78691253D0CD
:1051B1001251CE12542D806212803280E67F4474E7
:1051C10053201702744E7E0112910180157F4F7496
:1051D1005720170274457E011291017E08E51E12C7
:1051E10090E17E0EE51D1290E17E14E51C1290E126
:1051F1007E1A74641291017E21E51B1290E17E27D3
:10520100E51A1290E17E2D742E1291017E33E5197B
:105211001290E17E39E5180290E1742D2017027495
:105221002B7F707E151291011252397E3A12902213
:105231007E01904D3F02493C7E1BE51C1290E17EB0
:1052410021E51B1290E17E27E51A1290E17E2DE502
:10525100191290E17E33E5180290E17E097F271251
:1052610052BC1255181251661255632017171002BD
:1052710014121E0212879F120F1E1249D21251914F
:105281001298F880E9120EFF203026203128786626
:105291001253D01252E9786612547B78691253D0B6
:1052A1001252F5786912547B12542D12539B0254F9
:1052B100CD12572680F212804780ED79D48700C045
:1052C100011255DAD001A70009EE2406FEB9DBED83
:1052D1008700C217B82F02D217C001125597D0010B
:1052E100775F301702772F22751E007F447E0112EF
:0D52F10055A780107F4F7E011255AF7E083B
:1052FE00E51E1255F5F51E7E0EE51D1255F5F51D32
:10530E007E14E51C1255F5F51C7E21E51B1255F594
:10531E00F51B7E27E51A1255F5F51AA217926FC2E4
:10532E00177E2D12558F3017031253577E33E51902
:10533E001255F5F5197E39E5181255F5F518301791
:10534E000312537AA26F921722E51975F00AA4255B
:10535E001875F006A42405FBE435F0FC123D46EB6F
:10536E0075F00A84F51985F018025214E51975F0D6
:10537E000AA4251875F00AA4FFAEF07C007D061273
:10538E003C30EF75F00A84F51985F018227F707E97
:10539E001512559F7E1BE51C1255F5F51C7E21E559
:1053AE001B1255F5F51B7E27E51A1255F5F51A7EDB
:1053BE002DE5191255F5F5197E33E5181255F5F54B
:1053CE001822E6FD33921718860418860330170349
:1053DE00123DDE7A09792778C0123CD18B1EADD3EF
:1053EE00ACD2AB0679EA7860123CCF8B1DAF06AE1D
:1053FE00D27C177D70123C3D8F1CAF05AE047C0332
:10540E007DE8123C3D8F1BAF05AE047C007D64121F
:10541E003C3D8F1AED75F00A84F51985F01822E5DA
:0A542E0063FC339217AB62301703E2
:10543800123DD6305C0A7AD2123B327840123CD404
:10544800AE04AF037C277D10123C3D8F1CAF05AE28
:105458000480B178427B607CEA800678407B207CBF
:105468004E12810F79277810123CCF8B1CAF06AEF5
:10547800D28091E51E75F00AA4251D75F00AA425B1
:105488001C75F006A4251BFBE435F0FC7A0A123BD8
:1054980024EB251AFBE43CFC7A0A123B32EB251973
:1054A800FBE43CFCE43DFD7A0A123B44EB2518FB87
:1054B800E43CFCE43DFD301703123DDEA60518A6CA
:1054C8000418A603221254E8305C0A7A40123B32D0
:1054D80078D2123CD4301703123DD68C638B6222EB
:1054E8001254F87A0A123B24EB2518FBE43CFC2200
:1054F800E51C75F00AA4251B75F00AA4251AFBE41F
:1055080035F0FC7A0A123B24EB2519FBE43CFC221B
:10551800125541129A0DC20212554110000810018D
:105528000510021080F51031EF103004D23080E8F9
:10553800D23180E47F34024E48904D027F357E00A0
:1055480012496D904D18203009904D282031039054
:055558004D091F7E1744
:10555D0012493C0298F87F357E01904D3012496D0D
:10556D007F347E3A125666744E1291011298F812DB
:10557D009A0DC2027F347E3AD21775115975124EAB
:10558D00802675112E751227801E75115F75122FCD
:10559D00801675112B75122D800E75114E751253C7
:1055AD008006751145751257125666E511301702B2
:1055BD00E5121291011298F810000B10010810025B
:1055CD000280F50256611017E2D21780DE75112F99
:1055DD0075125A125666E8B4FF29745FD26E802395
:1055ED0075115F75125A80104430F81255FFE8544A
:1055FD000F22751130751239125666E8B4FF04E5A5
:10560D0011D26E547F1291011298F81000271001DB
:10561D000510023F80F5D26EB512004009B45F024D
:10562D00800FE51180DD04B43A04745F80D5B46059
:10563D00D2744180CED26EB51104E51280C55004EE
:10564D00E51180BF14B44004745F80B7B45EB474C8
:10565D003980B0F890567B8003905677C007EF24C1
:10566D0008FF129053D0070298F80205F8F80205CA
:02567D0000002B
:10983D0075A70090986F75F02D84C2D5C2D16017B1
:10984D00D2D1146007D2D514600DC2D1E5F093FCCE
:10985D00742D95F093FB22E5F093FB742D95F09309
:10986D00FC220009121B242C353E474F58606870AE
:10987D007880888F969DA4ABB2B8BEC4CACFD4D918
:10988D00DEE2E6EAEDF0F3F6F8FAFCFDFEFFFFFF8F
:1099DC00ED8BF0A430E70205F0C3E895F020D50438
:1099EC0025F025F0FEED8CF0A430E70205F0C3E97C
:0D99FC0095F030D10425F025F0FF02997C94
:109699002015437E1C7F5312997C7F5912997C1E99
:1096A9007F5712997C7F5512997C7E2312997C7F72
:1096B9005712997C1E7F5912997C7F5312997C1FEE
:1096C9007E2012997C7F5A12997C7E1E12997C7F8A
:1096D9005212997C800A7E1C7F5390971F129053D7
:1096E90030741CE5716018E57012983D781F795641
:1096F9007D091299DC3015031297090DBD16F32265
:10970900C0060E30D5021E1E12997CD0061F30D11C
:0F971900020F0F02997C070700386C446C380070
:108A45007F567E05128B787F3D128B8B7F6F128B45
:108A55008B7E1F7F41128BD17E0A7F41128BDC7E7C
:108A6500227F59128BDC20120122127A45857A1D4C
:108A7500855E1C857B1B855F1A7AC0C26F128BE8E9
:108A8500BAB7048C1C8D1D206F52128B537C007D50
:108A950014123C3074562F20D1029F9FFF24CB40E7
:108AA500028037EF248850028030EA1475F0038481
:108AB500FE12997CC3E51B957BFEE51A955F92D561
:108AC5005004EEF404FEEEC313FE24E0400C741FC4
:108AD5002E30D5029E9EFE12997CDAA1AC1CAD1DEE
:108AE500128B537C007D03123C30EFA2D17E047FB4
:108AF5005392D175F080305C04F5F08001A4A2E7B3
:108B050092D5E5F075F03284F8E5F075F00584C08E
:108B1500E0E5F0A2D533C0E0E860271290DAEE2454
:108B250006FED0E0F8D0E01290DAEE2405FE742CB3
:108B35001291010E0EE81290DA7E007F5474200225
:108B450090C2742B20D102742D12910180D0C3EDF7
:108B5500957AFFEC955EFE92D15003123DC6227EBA
:018B65003ED1
:108B660012997CDEFB227E0E12997C0EBE31F92212
:108B76007E0112997C0E0EBE41F8227E3312997C3C
:108B86000EBE40F9227E047D1112997C0E0E0EDD7A
:108B9600F81F1F7E35908BC8305C057E31908BCCDC
:108BA60002496D7405305C097E3274011290A3741B
:108BB600067E361290A37E3A74001290A37E3D0282
:108BC60090A33530300031363430007D0F12997C59
:108BD6000F0F0FDDF8227D0A12997C0E0E0F0FDDA6
:108BE600F7227803206F19127958127841E4F5F7C5
:108BF600C2B2C2B2E5F7D2B2C22064C07003D26F6D
:108C060022D8E1056DE56D2409F56D127841E4F58C
:108C1600F7C2B2C2B2ADF7F5F7C2B2C2B285F71B60
:108C2600F5F7C2B2C2B2E5F7FCD2B2C220543F3069
:108C3600E50244C0CC54C02323F51AE56D24F6F5AD
:108C46006D22206F19127958127841E4F5F7C2B2F5
:108C5600C2B2E5F7D2B2C22064C07003D26F220559
:108C66006D127841E4F5F7C2B2C2B2ABF7F5F7C2BE
:0E8C7600B2C2B2E5F720E4027B00D2B28087E2
:109607007E017F099096851290532051097E037F32
:1096170000743F029101E4FEFFC3E545128C84FD0F
:10962700940AED403D9464ED40027463128E4D7EC2
:10963700017F09E552240575F02D84AAF075F00520
:10964700A4CA75F00B842A9096709312983DBCB803
:10965700027BB87D04EE2DF8EF2DF90D1299DCDDB4
:10966700FB227E031290E180C6000C1622222D39C0
:10967700444F4F5A66707C7C87939EA9A9000909BD
:109687000800410000000000888000000000410041
:029697000800C9
:108C8400305D0A75F08AA42480E5F03400227F0068
:108C94002074137E0C908D1D1290537F0A7E0AE57A
:108CA4002E540F028E647E0BE571B4FF2DE5512422
:108CB400025003755100E551128C8475F005A4AC83
:108CC400F0FB123AFA7E0D781CE66004E61290DAA4
:108CD400EE2405FE18B818F48006128C84128E5304
:108CE4007F0C7E11E571602B0EE57064B460246422
:108CF400B475F03284C0F01290DACE2405CED0E000
:108D040075F00584C0F01290DACE2405CED0E023AD
:108D14000290DA90632A02493C0717FFFFFFCCE672
:108D240066BD5EAAA4EE6AB5F6AACDCE66FFFFFFC5
:108D340030744B78B979B7E6FC27FB1819E6FD3790
:108D4400F9EBF87B00123CD68B547F087E11A80601
:108D5400908D83129053E5542483E554500224FAF1
:108D640075F01984FB908D8B9328FEEB908D959371
:108D7400FD12997C0F0F12997C1F1F0EDDF3220345
:108D84000F0100FFFE03800000000007070D0C0B1D
:108D94000A05040302010102030405E57E700122B1
:108DA4007E007F35E57E128C84028EBE202C01224B
:108DB4007E197F36908DBE029053050EFFF0E01CA5
:108DC400F004F81CFFF02012457F15128B647F1FFE
:108DD400128B647F1720740DE53F20E0317E0190F3
:078DE4008E1302493C78BC2C
:108DEB00E66011E53F20E00C7E01908E1F12493C9E
:108DFB00E6028E64E53F30E00E7E06908E28305DF5
:108E0B0003908E3202493C22534541524348405312
:108E1B004154530043414C40414C5449005D203177
:108E2B0030404B4D2F48005D2035404B54530021B3
:0C8E3B0053455420484549474854210045
:108F4C00751900781DC2D5E630D50C1290DAEE24D6
:108F5C0005FE18B818F1227005B8191680EDD2D597
:108F6C003017E4CE24FBCE742D1290FDEE2405FEBA
:108F7C0080D574201290FD80D57F007E23AC5EAB33
:108F8C007A123ACC781DC2D5E630D50C1290E1EEAF
:108F9C002406FE18B818F1227005B8191680EDD207
:108FAC00D53017E4CE24FACE742D129101EE24069E
:108FBC00FE80D5742012910180D5123ACC781DC256
:108FCC00D5E630D5161290A3EE2404FE18B818F18D
:108FDC000E745E305C0274270290BE7005B81916D0
:108FEC0080E3D2D53017DACE24FCCE742D1290C289
:108FFC00EE2404FE80CB74201290C280CB123ACCAB
:10900C00781DC2D5E630D51912911EEE2408FE1833
:10901C00B818F10F0F0E0E7463305C027465029178
:10902C00017005B8191680E0D2D53017D7CE24F8C8
:10903C00CE740B12911EEE2408FE80C8740C129193
:03904C001E80C8BB
:1092B6007F797E24E55F30E70122AC5F1CAB7B1231
:1092C6003AFAE51B700E7420129101EE2405FE1287
:1092D6009304800C129304E51B1290DAEE2405FE2B
:1092E600E51A1290DAEE2405FE742C1291010E0E88
:1092F600E5191290DAEE2405FE745E029101742DD2
:10930600201702742B129101EE2406FE22E55F302F
:10931600E70122AC5F1CAB7B123AFAE51B700E74B8
:10932600201290C2EE2404FE12935D800C12935D0F
:10933600E51B1290A3EE2404FEE51A1290A3EE2478
:1093460004FE742C1290C20E0EE5191290A3EE24A0
:1093560004FE742A0290C2742D201702742B1290F8
:06936600C2EE2404FE2209
:1097B400E53724FD5001227E257F09A275E579C293
:1097C4006F6002D26F92D175F080305C04F5F08046
:1097D40001A4A2E792D5E5F075F03284F8E5F075BE
:1097E400F00584C0E0E5F0A2D533C0E0E8602712BC
:1097F400911EEE2408FED0E0F8D0E012911EEE2473
:1098040008FE0F0F205A2074601291011F1FEE24CE
:1098140004FEE802911E740C306F07740A20D10212
:10982400740B12911E80CB205904742E80DB2058B7
:0998340004746180D4746280D0D8
:1087B800E54424F64001227800E5520475F003846C
:1087C800F9E928FE24C45001FE1287F01287FC1E26
:1087D80012997CC3E998FE5003243CFE1287F01ED0
:1087E80012997C08B81FDA22EE2420FE24C2500316
:1087F8002402FE22E824F1E8C2D55006D2D5E8F4D6
:10880800241F23FF90887A93CF0493FAE545F5F067
:10881800A4ACF0FB123B5BE544F5F0A49BFBE5F050
:108828009CFCEB2420FBEC3400FC24F0500CEB24E3
:1088380060EC34009088CA93800EEB33FBEC33FC79
:10884800EB33EC3390889A93FAE5458FF0A430E740
:108858000205F0E5F020D502F4042A75F005201988
:108868000375F00384FF24DF50027F20C374329F16
:10887800FF22FF00FF03FA0BF318EA2ADE40CF5865
:10888800BE73AB8D96A880C068D64FE835F51BFD42
:1088980000FF00080B0E101214151718191B1C1DC9
:1088A8001E1F20212223242526262728292A2A2B71
:1088B8002C2D2D2E2F2F30313132333334343536A1
:1088C8003637373839393A3A3B3B3C3C3D3D3E3EFA
:1088D8003F3F4042444648494B4D4E5052535556EF
:1088E80058595B5C5D5F60616364656668696A6B63
:1088F8006D6E6F7071727374767778797A7B7C7D20
:108908007E7F808182838485868788898A8B8B8C09
:108918008D8E8F9091929394949596979899999A11
:108928009B9C9D9E9E9FA0A1A2A2A3A4A5A6A6A72C
:10893800A8A9A9AAABACACADAEAFAFB0B1B1B2B358
:10894800B4B4B5B6B6B7B8B9B9BABBBBBCBDBDBE91
:10895800BFBFC0C1C1C2C3C3C4C5C5C6C7C7C8C8D5
:10896800C9CACACBCCCCCDCECECFCFD0D1D1D2D222
:10897800D3D4D4D5D5D6D7D7D8D8D9DADADBDBDC77
:10898800DDDDDEDEDFDFE0E1E1E2E2E3E3E4E5E5D1
:10899800E6E6E7E7E8E8E9EAEAEBEBECECEDEDEE32
:1089A800EEEFEFF0F1F1F2F2F3F3F4F4F5F5F6F699
:1089B800F7F7F8F8F9F9FAFAFBFBFCFCFDFDFEFE07
:1089C800FFFFE54524FD400122E5520475F00384CC
:1089D800241FFE24C250032402FE128A1BEEFD242B
:1089E8001EFE24C250032402FE128A1BE544240200
:1089F80075F00520190375F00384F4042432FF246C
:108A0800EE500F128A10AE051E1E7C0512997C0EC0
:108A1800DCFA227F1512997C0F0FBF2DF822E5533F
:108A28000475F00384241FFE24C250032402FE129E
:0D8A38008A3B0E7F2312997C0FBF2DF9227F
:10913A0075A7007E007F2F9091D5129053205D1065
:10914A007E35746430190274A0128F0B20740F22BA
:10915A007E3974373019027455128F0580EEE54A4C
:10916A00B4040122B4060122E571128863EFFDE519
:10917A00700475F00384241EFE24C2401F24035089
:10918A001E9091C060099091C71460039091CEE43B
:10919A0093A3B4FF0122FE1291B480F32402FE7C51
:1091AA0004EDFF1291B40EDCF822EDFF12997C0F48
:1091BA00EF24CE50F7223B3C3D3E0001FF3C3D3EB2
:1091CA00010203FF3E3F01020304FF05387001104C
:1091DA00024007808001100340040060015003C070
:1091EA00070017FCA7FADFF43FE000A0024007805F
:109A3200AF177E00E53C128E477E0C742E12910108
:109A42007E12E53B128E477E1E742E1291017E24F9
:059A5200E53A028E4719
:10993D007F797E16743B1290FD7E18E53F128EB234
:10994D007F797E0078AEE6128EB27E0A743B12905D
:10995D00FD7E0CE53E028EB27F797E00E540128ED3
:0F996D00B27E0A743B1290FD7E0CE541028EB271
:10941F0075170078751294727453201702744E20CA
:10942F007406E52E54074430AF1712949C7E3BE52B
:10943F007DC4540F1290E12074077E07742012919F
:10944F00017878129472E5172409FF7457201702D8
:10945F007445207402742012949C7E3BE57D540F5A
:10946F000290E1E6FD339217188604188603301731
:10947F0003123DDE79177870123CCF8B13AF06AE17
:10948F00D27C007D64123C3D8F148D15227E00121C
:10949F0091017E07E513128E647E19746412910197
:1094AF007E20E514128E477E2B742E2073030E74CC
:0B94BF002C1291017E2FE515028E4754
:1091FA00C234E54A602890927B14601B90927F14D7
:10920A00601590928314600F90928714600990926F
:10921A008B14600390928F7F717E0012493C7F719C
:10922A007E002055052054068009745B8002745C18
:10923A0012910130262EC2267F687E0090929312E8
:10924A00493C7F66A85AE54AB4060108E875F06405
:10925A0084740AC5F084C0F012911EEE2409FED06F
:10926A00E012911E2008097F367E2E74411290C2A8
:10927A00222440260026402000244028002840209E
:10928A000024402900294020004D41524B00E53579
:10929A0024C85011E59020E20CD2347E237F7190CD
:0C92AA0092B012493C22455849543F0044
:10936C0020144F7405129A77EF33EE33F9EF0303A1
:10937C00541FF5F09093BFE993A4C5F013C5F013F7
:10938C00C5F013C5F013C5F0135403FCE5F013FB43
:10939C00E9242093C9244093C39BC4540FFBE99C3C
:1093AC00C4FC540FF9EC54F02B2446F57BE934F64D
:1093BC00F55F22FFFFFFFFFFE6C5AD9C8F857D7734
:1093CC00726E6C6A696A6A6C6F747A828D9DB4D99C
:1093DC00FFFFFFFAE9DCD3CEC9C6C3C0BEBBB9B729
:1093EC00B5B4B2B0AFADABAAA8A6A4A2A09E9C99EE
:1093FC0096918C00381CE735D137246F00C5B3C16A
:10940C00E61F66B60E68C21867AADBF4EDB946759E
:03941C0010A2009B
:109A5700D2A27408D2A1D2A300C2A3C2A1D2A300EA
:109A6700C2A3D5E0EF7405D2A300C2A3D5E0F822C4
:10003300C2A3D2A2D2A1D2A300C2A375F008339265
:10004300A1D2A300C2A3D5F0F5C2A175F003D2A338
:0700530000C2A3D5F0F82262
:10841800120033D2A300C2A3C2A175F008E4D2A30C
:1084280000C2A3A2A233D5F0F5FE75F008E4D2A3EA
:1084380000C2A3A2A233D5F0F5FFD2A300C2A322A3
:10844800E478806608B88BFB70012274D512841812
:108458007881C3EE13FEEF13F692D118EE2460F67E
:1084680074D61284187888EF33CE33CE33CE33CE19
:1084780033A2D192E25407FCEEFB7A08123B24ECBB
:10848800244FF608EBF674D9128418EF543F78821B
:10849800F67886EF33CE33CE33CE33CE335403F66D
:1084A80008EEF618161608E6C4FF54F0F618E6C4E7
:1084B800CF540F2FF674DA128418EF232354FC7864
:1084C80083F67884EEF608EF54C0F67880E4660800
:1084D800B88AFBF6221284207889C3EF96FF18EE3B
:0884E80096FEA2E79216501067
:1084F000123DC6740FF8F9123B71EF2CFFEE3DFEF2
:10850000788BEEF608EFF622E6182016072CF7E631
:108510003D19F722C39CF7E69D80F66A405E8056BF
:10852000E050F04B0044803DC0384031D02BA025B6
:10853000601F2018D00144015801680178018801AA
:10854000A001B401D001EC02100238026802A07848
:10855000BE8020858E8A9D8F4D95BA9A97A0BEA623
:1085600031AC53B22AB801BD6F128420788DEEF67B
:1085700008EFF67887798C123B71788379901285B1
:10858000087885798C123B71788179921285087808
:108590008DE624E4FE08E63392D13392D554FCFFF5
:1085A000EEA2D133A2D533FE780F7992123B7178C7
:1085B000947990C3EC97F61819ED97F67994908515
:1085C0001B7F197D0EEF93C3971F19EF93971F0918
:1085D0001DED600240EF0F908535798DEF93F7091F
:1085E0000FEF93F7788E7994123B7190854FEF934C
:1085F000C39BFB1FEF939C2440FC7897E62BF61857
:10860000E63CF618E436F67406129A77EEC20F606E
:0486100000FCEFFD7E
:108614007407129A77C3ED9FFFEC9EFE789CEF26B9
:10862400F618EE36F6222014347897799A12878257
:10863400123D2FEE24C0FE7C007D05123C0A8E61A3
:108644008F601295ED75C70375C6FE75B901E5BC5B
:108654002560F57AE5BD3561F55E1295FA7897796E
:108664009AC3E697FB1819E697FC7A02123B24207A
:108674000F0C7A02123B24ECFEEBFF028705A2E703
:1086840092D55003123DD6EC704EEBFE24D85048E0
:10869400789BE6A2E713FC08E613FBEC30E708300E
:1086A400D536123DD6800320D52E7F00EBFD123C3B
:1086B4003DBE0024EF20E72024E0501C789DE6FC1A
:1086C40008E6FB7AFF123B32EB2480E43CFBE43DFA
:1086D400FCEB2FF618E43CF6799CE77700FB19E7EE
:1086E4007700FCA2E792D55003123DD6799DE7FAB4
:1086F400123B32ECFBEDFC30D503123DD6ECFEEB25
:0C870400FF12872320140312876778956A
:108710007998E6F776000809E6F776000809E6F7A3
:10872000760022EE2408FE7403300F111295ED122C
:108730000622E5BF1295FAF4240623540FFD7C00AF
:10874000123B10789FE6FC08E6FBC374109DFA12FA
:108750003B32EFF8EEF9123D2FE878A02FF6FF1824
:10876000EE39F62480FE2292754003123DC6EF33A7
:10877000EE33F579C276307508E57924F15002D2EE
:108780007622E627FB1819E637FC1819E637FD2292
:108790001279D87F087871793A1287AB02337B85DA
:1087A0005E63857A62787379647F06E6F70809DF8D
:0887B000FA227864797380F16C
:103AAA00E4FEFFFC7D0A791DE7540F2FFFE43EFE7A
:103ABA00B91902800619123B1080ED301703123D26
:103ACA00C622305C2BEC3392175003123DD6EC24FD
:103ADA00D950047C277B007AD2123B32EB33CC33A9
:103AEA00CD33CC33ED33FBEC33FC301703123DD628
:103AFA00EC3392175003123DD67919123D46F70955
:103B0A00B91DF8A70322EFF88DF0A4FFEDC5F0CE9A
:103B1A00A42EFEEC88F0A42EFE22EB8AF0A4FBE58C
:103B2A00F0CC8AF0A42CFC22EB8AF0A4FBE5F0CCC2
:103B3A008AF0A42CFCE435F0FD22EB8AF0A4FBE524
:103B4A00F0CC8AF0A42CFCE435F0CD8AF0A42DFD4B
:103B5A0022EB8AF0A430E70205F0E5F0CC8AF0A463
:103B6A002CFBE435F0FC2286F0E7FDA4FAABF01951
:063B7A00E786F0A42BFB1E
:103B8000E435F0FC18E68DF0A42BFBEC35F0FCE4FA
:103B900033FDE687F0A42CFCED35F0FD22EB89F037
:103BA000A4CBAEF08AF0A42EFEE5F03400FDEC8943
:103BB000F0A42EFEE5F03DFDE433CC8AF0A42DFD0B
:103BC000E5F03CCEFC22EB89F0A4CBAFF08AF0A468
:103BD0002FFFE5F03400FEEC89F0A42FFFE5F03E66
:103BE000FEE433CC8AF0A42EFEE5F03CFCED89F037
:103BF000A42EFEE5F03CFCE433CD8AF0A42CFCE5D9
:103C0000F03D8E058C068F04FF22C2D5EC30E7050F
:103C1000B2D5123DCEEE30E70DB2D5123DC6123C04
:103C20003D123DCE8003123C3D30D503123DC622ED
:103C3000C3EC13C0E0ED132FFFD0E03EFEBC000B41
:103C4000BE0029EF8DF084FFADF022E4CCF975F0D1
:043C500008EF2FFF4B
:103C5400EE33FEEC33FCEE9DEC994005FCEE9DFE4C
:103C64000FD5F0E9E4CEFD22EDF9F5F0EE8420D293
:103C74001CFEADF075F008EF2FFFED33FD40079902
:103C84005006D5F0F222C399FD0FD5F0EA22EC33A9
:103C9400EE3400FEEF3400FF7D007A0079007809ED
:103CA400C3ED9AFDEE9BFEEF9CFFB392D54009ED68
:103CB4002AFDEE3BFEEF3CFFA2D5E933F9ED33FDDF
:103CC400EE33FEEF33FFD8D92279007A00C3801592
:103CD40079007A00C3EA13FFE913FEE8132BFBEE25
:103CE4003CFCEF3DFDE4F5D2F5D333FE7F19C3EE82
:103CF40098FEE5D299F5D2E5D39AF5D3B392D5409F
:103D04000DEE28FEE5D239F5D2E5D33AF5D3A2D5A6
:023D1400EB338F
:103D1600FBEC33FCED33FDDF0122EE33FEE5D2335F
:103D2600F5D2E5D333F5D380C3EDC454F0FEECC42D
:103D3600FF540F2EFEEF54F0FFEBC4540F2FFF225B
:103D4600EC75F00A84FCEB54F025F0C475F00A8497
:103D5600C4CBC454F025F0C475F00A842BFBE5F0FF
:103D660022AC10AB11123D46A904AD03FA7C197BB7
:103D760099123B24AE04AF03EA75F006A4F8AC1220
:103D8600AB13123D462875F00A8485F014F8EF2B24
:103D9600FFEE3CFEEF28FFE43EFEE43DFDE439FC89
:103DA60022CFC513CFCEC512CECDC511CDCCC510F1
:103DB600CC22C3E49FFFE49EFEE49DFDE49CFC222E
:103DC600C3E49FFFE49EFE22E4C39DFDE49CFC2227
:053DD600C3E49BFBE4C7
:103DDB009CFC22C3E49BFBE49CFCE49DFD2275D47C
:103DEB00107B807A0079807800EAF5F0A4FCADF0C6
:103DFB00EBF5F0A4FEAFF0EB8AF0A4C333C5F033C0
:103E0B00C5F092D52DFDC5F03EFEE430D501043F43
:103E1B00FFB5150DEEB51409EDB51305ECB5120193
:103E2B00224006EA98FAEB99FBD5D40ABB00012293
:103E3B000ABA00010B22C3E913F9E813F8EA28FACE
:103E4B00EB39FB80A478087B807D807C00EDF5F05E
:103E5B00A4FAE5F08EF0B5F007EA8FF0B5F0012289
:103E6B004003ED9BFDD827BDFF0122EDF5F0A4F932
:103E7B00A8F0ED04F5F0A4C399FAE5F09813CA1372
:103E8B0029F9E83AF8C3E99FE89E50010D22C3EBEC
:103E9B0013FBED2BFD80B67473F8F9123EB6754724
:023EAB00FFEF27
:103EAD0020E10513EE13F54722E627FA0809E63758
:103EBD00FB0809E637FC30E70AC3E49AFAE49BFBFA
:103ECD00E49CFCEA75F01FA4AAF0EB75F01FA42A80
:103EDD00E5F03400FBEC75F01FA42BFBE5F034008E
:103EED00FC903F0960020583EB93FE70037F022275
:103EFD007F01BC0106EB24AC50011F220000000025
:103F0D0000000000000000000000FFFFFFFFFFFFAA
:103F1D00FFFFFFFFFFFEFEFEFEFEFEFEFDFDFDFDB3
:103F2D00FDFDFCFCFCFCFCFBFBFBFBFBFAFAFAFACF
:103F3D00F9F9F9F9F8F8F8F7F7F7F7F6F6F6F5F500
:103F4D00F5F4F4F4F3F3F3F2F2F2F1F1F0F0F0EF43
:103F5D00EFEEEEEEEDEDECECEBEBEBEAEAE9E9E89A
:103F6D00E8E7E7E6E6E5E5E4E4E3E3E2E2E1E1E004
:103F7D00E0DFDEDEDDDDDCDCDBDADAD9D9D8D7D780
:103F8D00D6D5D5D4D4D3D2D2D1D0D0CFCECECDCC10
:103F9D00CCCBCAC9C9C8C7C7C6C5C4C4C3C2C1C1B1
:103FAD00C0BFBEBEBDBCBBBABAB9B8B7B6B6B5B464
:103FBD00B3B2B1B1B0AFAEADACACABAAA9A8A7A628
:103FCD00A5A4A4A3A2A1A09F9E9D9C9B9A999897FE
:103FDD0097969594939291908F8E8D8C8B8A8988DC
:103FED0087868584838281807E7D7C7B7A797877D4
:103FFD007675747372716F6E6D6C6B6A69686765D7
:10400D0064636261605F5E5C5B5A595857555453E7
:10401D0052514F4E4D4C4B49484746454342414006
:10402D003F3D3C3B3A38373635333231302E2D2C2F
:10403D002A29282725242321201F1D1C1B1A181768
:10404D0016141312100F0E0C0B0A080706040301A9
:10405D00FFFEFDFCFBF9F8F7F5F4F2F1F0EEEDEBF8
:10406D00EAE9E7E6E4E3E2E0DFDDDCDAD9D8D6D54C
:10407D00D3D2D0CFCECCCBC9C8C6C5C3C2C1BFBEAB
:10408D00BCBBB9B8B6B5B3B2B0AFADACAAA9A7A613
:10409D00A4A3A1A09F9D9C9A9997959492918F8E80
:1040AD008C8B898886858382807F7D7C7A797776F3
:1040BD007473716F6E6C6B696866656362605E5D6B
:1040CD005B5A5857555452514F4D4C4A49474644E7
:1040DD0043413F3E3C3B393836343331302E2D2B66
:1040ED00292826252322201E1D1B1A1817151312E9
:1040FD00100F0D0C0A08070504020101C21DC23282
:10410D00752C00C3E5679576FBE5689577FCE56949
:10411D009578FD30E705D261123DDE24F050031293
:10412D0041DFAA07A906123BC6EC2401FCED3400C1
:10413D00FDEE3400136002D232ED13FAF519EC13D3
:10414D00FBF9F51AAC02123B9D8B128C138D148E5C
:10415D0015C3E5649573FBE5659574FCE56695758A
:10416D00FD30E705D262123DDEEBF9F51FECFAF5F5
:10417D001DED6002D23230320122123B9DEB251231
:10418D00F512EC3513F513ED3514F514EE3515F573
:01419D00150C
:10419E0040E1123DE9EB242E40D9EA2401CB340054
:1041AE00FC7A07793D123B9DC010C0118E108D1107
:1041BE008C128B13E4FCFD7E077FD0127058851293
:1041CE0003851302D011D010BB0005BA0002D21D18
:1041DE0022B261C374809BFB74F59CFC74209DFD20
:1041EE0022302A0578A8760022E54824F6403EE5DE
:1041FE005804603975A700758307E559C42408F57E
:10420E0082E070290582E0FF120631C3E5BD9F40B2
:10421E001C205206D25278A8762343820FE0642FD8
:10422E00600BC3E559955850040559C25222E55802
:10423E00B4FF012285581175A704758307E548243C
:10424E00F650028064201261202905202A0280592E
:10425E00787379AF1287A9E4F516F5177510001269
:10426E0042D0E51070031287B21242E9302910E5F0
:10427E001B2517F517F51BE51C3516F516F51C1243
:10428E0042F41287B20510C3E511951050D175A7EF
:10429E000078AF79730287A9E55AF51124F6500319
:1042AE0075110A75A7047583067510001242D01297
:1042BE0042E91242F40510C3E511951050EE75A7B0
:0242CE000022CC
:1042D000E510C4F582E0E0F564E0F565E0F566E040
:1042E000F567E0F568E0F5692205A71244B9122BDD
:1042F000F105A722E9F0E51CF0E51BF022E510C46A
:10430000F582E0F512E5822406F582E0F511E0F58C
:104310001CE0F51B2220282DE558B4FF012275A7CB
:10432000047583078559101242FDE0F513E07F7A8A
:104330007E3D1290C2E5137E391290C2E5127E35A1
:104340001290C2802875A704758306855B101242FF
:10435000FDE512700B7E3A7F79745D129101800D3C
:1043600075F06484E5F07E397F7A128EFFE5116482
:10437000B4601EE51112983D781F79567D167A1D9E
:10438000E53F20E0047D187A1F1299DC0DEDB5029F
:10439000F8751619751779E51C24ED402BAE1CAF86
:1043A0001B1244837C007D32123C3DC005EFAF17E9
:1043B000AE16128EB8CE2405CE742C1291010E0EBC
:1043C000D0E023128EB2801B12447A1243F5CE2421
:1043D00005CE742C129101CE2402CEE875F005842E
:1043E0001290DACE2404CE7422305D0274661291EB
:0643F0000175A70022EE9A
:1043F600243D50047EC37F4B7C017DF4123C3DC0BE
:1044060004C005EF6007AF17AE16128EB8D007D0FE
:10441600067C007D32123C3DA805EFAF17AE16CEE6
:10442600240ACE0290DA12447AEE2450305D03EE6E
:1044360024A150047EC37F4B7C017DF4123C3DC019
:1044460004C005EF6007AF177E2F128F05D007D087
:10445600067C007D32123C3DC005EFAF177E371259
:1044660090A37E3B742C1290C27E3DD0E075F00581
:10447600840290A3E51B2402FFE4351CFE305D1A7E
:10448600BEC305BF4D028012AC06AB077A1B123BBA
:10449600327832123CD4AE04AF03227873796412B8
:1044A6003EB6124109751CC3751B4B2032048B1C8A
:1044B6008A1B221244A130320122AC19AE1AA91D60
:1044C600AF1FB90005BC00028010C3E913F9EF1352
:1044D600FFC3EC13FCEE13FE80E8BF29005006BEB6
:1044E6002900500122C3EF13FFC3EE13FE80EB7CBD
:1044F600C6C6C6C6C6C6C6C67C18387818181818E2
:1045060018187E7CC6C60C183060C0C6FE7CC6C6AF
:10451600061C0606C6C67C0C1C3C6CCCFE0C0C0CA1
:104526000CFEC0C0C0FC0606C6C67C3C66C0C0C049
:10453600FCC6C6C67CFEC6C6060C18303030307CBB
:10454600C6C6C67CC6C6C6C67C7CC6C6C67E0606AB
:1045560006CC78000018187E7E18180000000000AF
:10456600007E7E0000000000000000000000000049
:1045760000000000000000000000008080A0C0A035
:1045860000304020C08080C0A0A0000060A0600075
:1045960000A040A05098D090882050A850888850FD
:1045A600A8502060806000000040E040000000004D
:1045B60000800000E0000000000000400020408075
:1045C6000040A0A0A04040C04040E0C02020C0E085
:1045D600E0204020E02060A0E020E0C02020C06075
:1045E60080E0A0E0E020404040E0A0E0A0E0E0A0C5
:1045F600E020C0004000400000800080002060E015
:10460600602000E000E00080C0E0C080E0E0E0E084
:10461600E0000000000040A0E0A0A0C0A0C0A0C034
:1046260040A080A040C0A0A0A0C0E080C080E0E084
:1046360080C080806080A0A060A0A0E0A0A0E04034
:104646004040E0202020A040A0A0C0A0A080808004
:1046560080E0A0E0A0A0A0A0E0E0E0A040A0A0A094
:1046660040C0A0C0808040A0A0C060C0A0C0A0A0E4
:1046760060804020C0E040404040A0A0A0A060A0D4
:10468600A0A0A040A0A0A0E0A0A0A040A0A0A0A0A4
:10469600404040E0204080E02020A870202070A804
:1046A600202008F030D0100000F0A8A8000000E09C
:1046B600000000902048708898984000E0E0E000F4
:1046C60060909090909060206020202020706090F4
:1046D60010204080F06090102010906010305090B4
:1046E600F01010F080E010109060609080E09090E4
:1046F60060F0102020404040609090609090606094
:104706009090701090600000000000000000000013
:1047160000000000506050007070500000788070FB
:1047260008F000F8888888F800C0C810204098185B
:1047360000C0B098B0C000602040000000000090AB
:10474600D8FCD8900000246CFC6C24000020A870D3
:10475600A82000002020F820200000000000000013
:0D47660080000000F00000000000000000D6
:10477300606000081020408000708898A8C8887086
:1047830020602020202070708808102040F8F81046
:10479300201008887010305090F81010F880F0083E
:1047A300088870304080F0888870F80810204040F6
:1047B30040708888708888707088887808106000D6
:1047C3006060006060000000800000800000204006
:1047D300F84020000000F800F80000002010F81056
:1047E3002000708808102000200000000000000056
:1047F30070888888F88888F08888F08888F07088BE
:104803008080808870E09088888890E0F88080F0CD
:104813008080F8F88080F0808080708880B88888F5
:1048230078888888F888888870202020202070382D
:104833001010101090608890A0C0A0908880808095
:10484300808080F888D8A8A88888888888C8A8988D
:10485300888870888888888870F08888F08080804D
:1048630070888888A89068F08888F0A090887088FD
:104873008070088870F8202020202020888888886D
:1048830088887088888888885020888888A8A8A8FD
:10489300508888502050888888888850202020F8A5
:1048A3000810204080F800CCAC9CACCC0000CCD4E9
:1048B300E4D4CC0004781828C800FC40A040182099
:1048C3002018000000000000F800000000A040A035
:1048D3000000006000606000600060006060000035
:1048E300F0A8A8A8A8705070000000005090B890DD
:1048F300D0908860505000707050F888B898B8888D
:10490300F8304C5C6060603C00E0F0080808F88018
:1049130088482818F804008820208870000080C088
:0B492300A090F8000080A0D0A8F400D5
:030000000200619A
:03000B00027C3341
:100010007F797E00E581128EBE1298F8129A11E463
:10002000F537F534F520F52FC229C22AC268C22758
:03003000021F9C10
:06005B00752EF0021DBE2F
:107C3300C0D0C0E0C0F0C0A775A700C083C08275E4
:107C4300D008758A3D758CEA0532E532700215322B
:107C53000530E530640A6023E531B40C0BE530B43C
:107C63000106127F3112936CE531B4180BE530B481
:107C73000606127F3112936C027DE5C2AFD2C07546
:107C8300C07AD2AFF5300531E53164197030F53182
:107C9300C22C7D0A7404129A77EE24F54014240250
:107CA300400E24014008202005DDE9021DD8D2251D
:107CB300D22CE5A6600215A678A9E6600116E53187
:107CC300B40206201A0312956B206A1A301017307B
:107CD3007414E53724FD400EE536700AE59020E084
:107CE30005753612D22E302E09E5367005C22E12D6
:107CF3007EB8E5366002153678A8E66001160535CC
:107D0300E53570021535E590307A0B30E108D2780D
:107D1300C27AC201800C307B0930E206D279C27B81
:107D2300C202E59044F8F4700B753500302D05C29E
:107D33002D127EB8E53360041533806DE590F4545D
:107D4300076066F52075330820100375A6FF78A831
:107D5300E67056202D53202E50301004E53670491E
:107D630020100C201109E53524F55003753304D296
:0F7D73001BD2A5D2A675B40C75B22278A776558F
:107D8200C21C053420272320682020291D202A1AFE
:107D9200A21072115014A2017202500EE53424385E
:107DA2004008200116D27B7534C8E5317015129A4D
:107DB2005774E8120033801B027E5EE53770EBD207
:107DC2007A80E475F00384E5F070ED1284DD74E8E6
:107DD200120033E531B40C0312862AE531B41803DC
:107DE20012862A78A8E67019201005201106802133
:107DF200E536700DE59020E218E53524B45012D234
:107E02002DD2A6201002C2A6D2A57418127EAB8073
:107E12001C20340E305A08E54A603C1414603812B3
:107E22007EB8101B08A25892A5A25992A675A70067
:107E3200D082D083D0A7D0F0D0E0D0D0202006C509
:107E4200A66003C5A632201003021DD87581DB741B
:107E520010C0E0E4C0E032127E7680C6C218B402DE
:107E620002D21812856930180874E4120033027DB8
:107E7200D5027DD078A7E66002162230754079AA35
:107E82007700E579602C14FF760D24CE4006EF9042
:107E92007EFF93F6301C1FEF249C7410400BEF24DE
:107EA2000A75F0DFA4746F95F0C21CF5B4C313F524
:0E7EB200B22278A7767DD21CE4F5B4F5B22298
:107EC000E57924CE50097628301CED741480DC79D5
:107ED000A1E5799740E2E57979AAC7272464200EC5
:107EE00003F4242CFF301C06EFF6243680BDEF206F
:107EF0000D02C313F6EF300D022436D21C80AE788B
:107F0000726D68635F5B57534F4B4845423F3C3946
:107F1000373432302D2B2928262422211F1E1D1BE9
:107F20001A19181716151413121110100F0E0E0D22
:107F30000DD2B5C28EAE8DAA8DAF8BAB8BE4F58D15
:107F4000F58BD28E30140122300C05E4FEFAFFFBD3
:107F50007C007D0A123B107C007D5E123C308F7EDF
:107F6000EE6003757EFFEAFC7A33123B24EBF5F0FA
:107F7000A4E5F0CB8CF0A425E0C5F035E0CB926C05
:107F800025F050060BBB0002D26C30E7060BBB009D
:107F900002D26CECF5F0A42BFBE5F03400FC306C65
:107FA000010C78A6E6C39BFF18E608F6EB18F61856
:107FB000E69CFE18E608F6EC18F6301401227A006A
:107FC00050040A123DC67C007D6E123C308FF07862
:107FD000A2E6A4FBACF0123D46EBBA0002F404FAB0
:0C7FE000E4F8FFEA30E70118E5796006DC
:107FEC002075031FF4042AF579EF38D27520E708C1
:107FFC0060037579FF028774C2750470F5E579F436
:10800C000460EFF57980EE12063178A2A6BE120656
:10801C002C85BC2B85BD2112062778A1A6BC120687
:06802C0022789DA6BE2291
:10006100D2B4D2C075C07AD22075A6FF75D75075AB
:10007100AE1375AF017581DB75A882D2BC7589514C
:10008100D28C7590F875EFBC75FDFFC258D259C27C
:100091001E78FFE4F6D8FDD2A47F64129A19C2A497
:1000A1001277B2129A57128453C22012956B129A88
:1000B1008B121C957F417E00901CD812493C7F52C7
:1000C1007E02901CC012493C1298F81236E6129832
:1000D100F8129A0DD2347450127EAB129A0D127E20
:1000E100B81232241297281298F8129A0D753A0014
:1000F100121E02E53A7006752EF4021DBE1232245C
:10010100128013121C8B1298F8129A097520001292
:100111008448121C8B7F787E00901CCB12493C7F57
:10012100427E0E78ADE6128EB27E17742E129101C8
:100131007E1B18E6128EB27E24742E1291017E2847
:1001410018E6128EB27F4C7E0E78AEE6128EB27E2B
:1001510017743A1291017E1BE53E128EB27E247411
:100161003A1291017E28E53F128EB27F56128B6CB6
:100171007F5A7E0B128F891290227F647E12129217
:10018100BA1298F81000161001161002613098F496
:10019100C298E599B4E0ED12325A020110021DD85D
:1001A100021F7422E53524D250F9E59020E2F4D003
:1001B100E0D0E0129A8B7F097E0030271F306B1C44
:1001C1009001D212493C1298F8123A2F124E5880DF
:0C01D1001D5550444154494E472E2E004D
:1001DD00129A8BE4FEFF9010A712493C1298F81268
:1001ED009A09C214C227C268E4F535F520753701A6
:1001FD00C26E900227120E6E900209730200FE026B
:10020D00110F024B7902093302094B020A05020B49
:10021D00C7020C390223940202902145584954011A
:10022D004C4F47424F4F4B20686901574159504F32
:10023D00494E54530157415950542D44495354017B
:10024D0057415950542D53454E44015254452A2F70
:10025D0054582F525801524F5554452D494E530164
:10026D00524F5554452D4F52440153455420484546
:10027D00494748540153455454494E475368690002
:10028D00123872E4F535F520753702C26E9002CE44
:10029D00120E6E9002A4730201EF02031C0203946E
:1002AD000202900206AF02070702065702029002F1
:1002BD00046C0202900234BA023667023717020448
:1002CD000D214558495401564152494F2020686926
:1002DD000158432D53455420686901014C4F43414A
:1002ED004C2054494D4501554E495401434F4D0144
:1002FD000144454C40414C4C40575054010154452C
:10030D005354464C4947485401010000123872E4D9
:10031D00F535F520753703C26E900348120E6E90B9
:10032D0003307302029002048D0207CE02049C0278
:10033D0004AB02081E0208F602050821455849546F
:10034D0001564152494F4241520153494E4B54407F
:10035D002D0153494E4B2D4D4F440153494E4B2DBD
:10036D00494E560154454320202040303040250051
:10037D0054432D564152494F014455414C53454E1E
:10038D00534F5200123872E4F535F520753704C21B
:10039D006E9003BA120E6E9003A8730202900204BF
:1003AD00BA0204C902077E0208AB0204D8214558DF
:1003BD004954014155544F43454E5401474C444512
:1003CD00504154480143594C5221302E01452F477D
:1003DD0046202020202E01494D50454C4C455200C1
:1003ED00123872E4F535F520753704C26E900407A6
:1003FD00120E6E9004047302029021455849540068
:10040D00E4F535F520F537C26E90042F120E6E907F
:10041D0004207302029002045402045902045E0285
:10042D00046321455849540152442D454501524418
:10043D002D464C41534801474838300144454C2026
:10044D00414C4C20464C0012398E80B4123901803B
:10045D00AF12387D80AA12046880A51277C82212C7
:10046D000FC81298F810001510010280F87F487E11
:10047D00059001D212493C1298F8123A0B020290E3
:10048D007F0AA20A1204F0920A1204E702031C7FEB
:10049D001CA20D1204F0920D1204E702031C7F251D
:0504AD00A20E1204F094
:1004B200920E1204E702031C7F0AA2081204F092B1
:1004C200081204E70203947F13A2091204F09209AE
:1004D2001204E70203947F2EA20C1204F0920C1273
:1004E20004E702039412062C8521BD0238728F1F85
:1004F200921712064F12062C85BD21AF1F1F7E399F
:10050200125587A21722300F087512001205268095
:10051200107F3F7E0390061612493C1298F8129AF9
:100522000902031C75A6FF129A8B1205E1740712C9
:100532009A778FF07406129A77EF2512C395F0A27C
:10054200E7926F4010FD24C050027D3FAC05C3749A
:100552003F9DFD800FF404FD24C050027D3FAC0599
:1005620074402DFD7F40128B647E1712997C0EBE63
:100572001EF91F306F020F0FEF6D70EDE536700A36
:10058200753606EC2513F5148C131205A41298F88F
:1005920010000710010830028B2215128086051206
:1005A20080827F377E28742E1291017F347E2174DF
:1005B2000A306F010412911EE514FC249C50027C47
:1005C20063EC75F00A84C0F07F347E2D12911ED048
:1005D200E07F377E361290E17F437E1E028F897F55
:1005E200057E09901CB312493C7F6B7E019005FF8A
:0705F20012493C7F757E02F7
:1005F90090060B02493C4455414C2153454E534FFB
:100609005200544543484E4F4C4F4759004E4F54A2
:100619002150524553454E540075C6F7802175C681
:10062900F8801C75C6F9801775C6FA801275C6FB65
:10063900800D75C6FE800875C6FF800375C6FD75F9
:10064900C70375B90122743F1290C20298F87F3727
:1006590012064F120631A8BC10000810010510023D
:100669000F80F508E824FD5002780012067E80E824
:1006790088BC02028D900697E8600990069F146075
:10068900039006A77F367E1B12493C0298F8202169
:100699002039363030002021353736303000495284
:1006A9002135372E36007F2512064F7E2A121E026B
:1006B900120631A8BF1206E410001210010510023B
:1006C9001580F508E824E750EC781880E818E83038
:1006D900E7E3780080DF88BF02028D7F247E27E56B
:1006E9003D28240C75F01884E5F0128E477E33748A
:1006F9003B1291017E35E53E128E470298F87F2E16
:1007090012064F12062C85BC2B1207411000081047
:10071900010510021780F2105C07205D0BD25C8086
:10072900E8105DE5D25D80E1D25C80DD12062C85A2
:100739002BBC8521BD02028D205C10205D1890071D
:10074900647F2D7E2312493C0298F8900778205D3A
:10075900F090076B80EB90077180E6406340204B77
:1007690063004654204B6300406340204E4D0046D1
:1007790054204E4D007F1C12064F120631A8BD129F
:1007890007AB10000810010D10021280F218B8FF13
:10079900EE783180EA08B832E6780080E288BD0256
:0B07A9000391E8237F1B7E29128C8443
:1007B400128E477E359007C8305D039007CB1249EF
:1007C4003C0298F83022003066007F1312064F1264
:1007D4000627A8BCE81207FF1298F81000101001B1
:1007E4000510021280EE18B8FFEA783280E608B8E5
:1007F40033E2780080DE88BC020319305C01237F79
:10080400127E2975F00A84C0F0128E4D7E35742E46
:10081400129101D0E07E3A0290E17F2E12064F122F
:100824000631E5BE7F2D7E2C1255F5F5BE02031967
:10083400120741120631A8BC02067E12062C85BDA1
:10084400217F09A20A12089F7F1BA20D12089F7F15
:1008540024A20E12089F120627E5BC1207FF1206F7
:1008640031E5BE7F2D7E2C1290E122120622E5BFD7
:1008740002092C120631A8BD1207AB120627E5BDEA
:100884001208DE12062C85BD217F09A20812089FDA
:100894007F12A20912089F7F2DA20C744E4002748D
:1008A400597E3A029101227F2512064F7E351206A7
:1008B40027A8BDE81208DE1298F810000810010DF0
:1008C40010021280EE18B809EA787880E608B87940
:1008D400E2780A80DE88BD0203917F247E2975F0C8
:1008E4000284C0F0128E4DD0E075F005A47E3B0268
:1008F40090E17F3712064F120622A8BF200F02781C
:1009040003E812092C1298F810000810010D1002C7
:0B0914001280E918B800E5780480E1CB
:10091F0008B805DD780180D988BF0203197F367EBC
:10092F003B0290E1D26875480A121E02D214121EC1
:10093F001D124B6D1225BB1201A580F5D214123179
:10094F004775150112500275B901E5BC04601C1200
:10095F00511675A6FF125166120F931298F8124A8C
:10096F005610020F5005124B3580E70515E515247B
:10097F002050D10201EFE55820E70A0559C39559D8
:10098F0050037559FF22E55820E70B1559E55964B7
:10099F00FE700385585922E55920E711D26B75A7D0
:1009AF0000758307E559C4F582E0B2E7F0220548E8
:1009BF00E548640A7002F54880131548E54864FF5E
:1009CF0070037548098006754800121E1D121E29F6
:1009DF0012423C129A8B120F0E900CF912628D126A
:1009EF0062401298F81000D21001C310020280F575
:1009FF00121E29E55822D2141209D620E703020A43
:100A0F00A3123147129A8B120F93900D1912628D08
:100A1F001298F8C29810021FE55830E7F83098F591
:100A2F00120B7B7E207F005011900D2F12496D12FB
:100A3F0098F8129A0980CA0201EF1B8B139001D20A
:100A4F0012496D1298F8C26B7B007514BC120DFE23
:100A5F001250E51250975025A814E824344004A6EC
:100A6F000105140BC3E5139B50E678BC120E403002
:050A7F006B03124E584C
:100A8400121E2912423C8084125048E51660E6D2B8
:100A94006B125142C003125019D003A91580C4C26D
:100AA4006B7559FF12423C129A8B120EFFE55930B6
:100AB400E703120F0E900D3912628D12625E1298C6
:100AC400F810000810010A10020C80F51209858044
:100AD400D612099580D11209A6E55930E7C9306BC1
:100AE40003120DC2121E29E558047003020A1012E3
:100AF400423C129A8B120F0E900D0312628D1298C3
:100B0400F810000810010510020780F5120E148079
:100B1400D3123147129A8B120F6D900D0E12628D03
:100B24001298F810000510021880F8120B48900D66
:100B3400245003900D2F12628D1298F8129A098096
:100B4400D00201EF12954274521294E57454129437
:100B5400F7E55804755900129531124A0C401612E3
:100B64004FDA125116124A56400B0559C3E55895EF
:100B74005950ECC322D32212989DC5F060F7C5F0FA
:100B8400B440F41298A2B440031298A2B452E6F509
:100B9400381298A2B454DE1298A2FA60D824EF4016
:100BA400D41298A2E53870CD1298A21298A21249D4
:100BB400F67B00124AC440BD1250F50B1249F6DA16
:100BC400F2C322121E02D2141209D6854849D22732
:100BD40075480A121E1D12423C129A8B1261E8904B
:100BE4000D44202903900D4F7E207F0012496D1281
:0D0BF40098F8C26A1225BB1201A5106A0212
:100C010080D7C227124FDA854948120DAA121E2930
:100C110012423C129A8B120FAD904CB33057039095
:100C21000D6512628D1298F810000510020580F80A
:100C31000201EF30579B80F0D2141209D630E7033E
:100C41000201EF1201A5121E2912423C85594912D7
:100C51009A8B120F0E900D4F12628D12624E1298E6
:100C6100F810000810010A10020C80F5120CC48063
:100C7100DB120CD180D6129A8B120F0E900D5A12E4
:100C8100628D12624E1262521298F8100008100121
:100C91000A10020C80F5120CDD80DB120CEB80D601
:100CA100120D70121E2912423C129A8B120FAD9036
:100CB1004CB312628D1298F810000510028580F86D
:100CC1000201EF0559C3E5589559500375590022A2
:100CD1001559E55964FF7003855859220549D3E533
:100CE100491495584003754900221549E54964FFA7
:100CF100700585584905492253454C21524F555499
:100D0100450021405245564552534540002140532C
:100D1100454E4440525445002140524543454956B1
:100D21004540002020404F204B4020202100202022
:100D31004641494C20202100214044454C40575018
:100D4100545300214053454C404C495354002053C7
:100D5100454C40575054402100204E455740504F7C
:100D610053402100405254454046554C4C210012FD
:100D71000E4FE55924CCF88602E54924CCF9986058
:100D810013146010500F18E608F618E86970F7A7F9
:100D910002120E3E22E559640F60F91908E618F6B1
:100DA10008E86970F7A70280E8120E4F78CCC257A5
:100DB100E6B4FF02800708B8DCF6D25722A61580F8
:070DC1007C78BC120E51E426
:100DC800F9F5A7758307E9C4F582E030E70AE92455
:100DD800BCF82434400276FF09C3E5589950E7125D
:100DE8000E0978BC79CCE6B4FF028002F70908E85E
:100DF800243450F2804079BC77FF09E9243450F854
:100E08002279CC77FF09E9242450F822120E4FC228
:100E18006F78DBB6FF04A900D26F18B8CBF5206F46
:100E28000279DC1978CCB6FF0122C3E8995007C6CD
:100E3800C7C6081980F478CC120E601251541251AA
:100E48005412515402515478CC120E60125130127F
:100E5800513012513002513075C703E54875F0041E
:100E6800A42480F5C622129A8B12492EE537602BEE
:100E780014602514601A14601214600A1460028049
:100E88001A1208AA8015120877801012083F800BE2
:100E980012083412365280031236701298F8129AD9
:100EA8000D120EFFD234E4F5B4F5B2A81F08E81409
:100EB800C26DB51D02D26D75F007206E0375F0097D
:100EC800A4FF206E010F7E007420306D02743E1264
:100ED80090C2D8DA1298F8E51D10000810010D101C
:0A0EE800021080C0651F60BC051DEC
:100EF20080B860B6151D80B275F003A422120F5A95
:100F02007E34900F0A02496D53454C00120F5A7EEF
:100F120031900F1902496D4E455854007F7B124E95
:100F22003880EC7F72120F5C7E2D900F3202496D79
:100F3200535441525400120F5A7E2A900F430249D1
:100F42006D40425245414B00120F5A7E31900F556F
:100F520002496D53454E44007F7B124E387E057424
:100F62005B1290BE7E1D745C0290BE7F7B7E009001
:100F72000F8212496D12314712317A7E1402496D85
:100F820053454E44202020202020202045584954FB
:100F9200007F7B7E00900F9C80D820202020202084
:100FA20020202020202045584954007F7B7E00903D
:100FB2000FB702496D455849542020202020202097
:100FC200204E455854007F7B7E05900FD202496D1A
:100FD2004E4F202020205945532020202020202021
:100FE20000D214E4F56CF56BF9FAFBFCFDFEC26F5E
:100FF200120645E5BD54F07013E5BF54F0700DE5DF
:10100200BC65BE7006E5BD65BF600122756A00124F
:1010120079D8E570D2E2B4FC3FC3E57199403970EA
:1010220023E5729A4032701CE5739B402B7015E5E4
:10103200749C4024700EE5759D401D7007E5769EF8
:1010420040167000A971AA72AB73AC74AD75AE761E
:10105200856C6F856B6ED26F127928E56C456B706B
:10106200AB306F36856F6C856E6B756A20E4FEFF60
:101072001279D812790DE57F6006DFF4DEF2801A6C
:10108200E56A600512790D80F7856EBC856FBD85B6
:081092006BBE856CBF123872C1
:10109A0080031277C8223E214558495400204558FA
:1010AA00495400127A59120645E5BDF55EF56CE51C
:1010BA00BCF55FF56B756A007561FF75A70490074B
:1010CA00001279F1B4FC12E582C313F561E56CF004
:1010DA00E56BF0E58260168005B4FF02800F127995
:1010EA0055E56C655E70DAE56B655F70D475A700CF
:1010FA0022E560758307C333F582E0A3F56CE0F55A
:10110A006B756A0022120FE3D214C22F1210AD754A
:10111A006000E561B4FF26129A8B9011397F0A7E2E
:10112A000512496D1298F87E08129A130201EF4CC3
:10113A004F47424F4F4B20454D50545900C210C2A1
:10114A0011129A8B120EFF302F0C7F077E0090101F
:10115A00A012496D80647F007E01C3E560128F0B87
:10116A007E0E74281290BE8560487407F51FFF7EB4
:10117A0000743E1290C2E5481210FD1287901217B1
:10118A00220548C3E5619548FD401CE51F2407F583
:10119A001F24C850E17F387E01ED04128F0B7E0EAA
:1011AA0074291290BE800DE51F2407FF7E0190105E
:1011BA00A712496D202F031217651298F81000190B
:1011CA0010012C10020280F51201A5302F560201DF
:1011DA00DD102F02D22F021147E56160F4E5606548
:1011EA00617005202FF080E9202FE6056080E7E591
:0911FA006160DEE56065617005CD
:10120300202FD58009202FD5E560700280CA156094
:1012130080CB2145584954015245504C4159015303
:10122300454E440144454C455445001210AD12103F
:10123300FB128790121851756A101279D812190887
:10124300D26E90121512492E120EA99012527302E9
:10125300114702240102127B02125E120FC8129878
:10126300F81000C710010280F81210FB1279F1C2C6
:10127300E2FF12787C02110F1210FB128790753770
:1012830000C26E9012B7120E6E9012907302122E5D
:101293000214DB0214E002127B0213310213360242
:1012A300127B021371021375021379021380021366
:1012B30084021388214558495401544E4320312355
:1012C3002035374B01544E4320312320392E36012C
:1012D30001505743403130234035374B015057437A
:1012E300403130234031394B01014D5850403130AA
:1012F300234035374B014D58502034232035374B8D
:10130300014D58502031232035374B014D58504063
:101313003130234031394B014D5850203423203193
:10132300394B014D58502031232031394B001231B4
:10133300A8800312319D780A12145974041294F58B
:1013430012149812952A1214B21279D8127A04122E
:10135300790D127B2F1215CAD5150C75150A1214A7
:10136300C51216E012952AE57F70DE02122E780A66
:1013730080067804800278011231A8800D780A80F3
:101383000678048002780112319D121459740412F4
:1013930094EA121498E5481294D1742A1294F7121D
:1013A30094F71294F712952A1214B21279D8127A7A
:1013B3000412790D127B2F1215CAD5154A854815CB
:1013C3001214C5E51C1294D1E51B1294D1E51B251B
:1013D30048F51BE4351CF51CE4A27792E7A274924E
:1013E300E0A27392E11294D1AD75AC74AB73787DC6
:1013F300E6C4121411AD78AC77AB76787DE612149F
:10140300111216FE12952AE57F70A002122E540FB8
:101413002375F00584F8C3EB33FBEC33FCED33FDAC
:10142300C3EB33FBEC33FCED33FD20E713EB28FB7D
:10143300E43CFCE43D1294D1EC1294D1EB0294D140
:10144300C3EB98FBEC9400FCED94001294D1EC12E6
:1014530094D1EB0294D18848120F38E4F54AF54948
:10146300756A207515011279D812790DD5150E8577
:101473004815E5492401F549E4354AF54AE57F7005
:10148300E574401294E574781294F774631294F738
:1014930074100294EA1216971216BCE53F1294EAEE
:1014A30074011294D1E54A1294D1E5490294D11200
:1014B30010FB756A20E4F51CF51BF514F51375157F
:1014C3000122753800E5141294D1E5131294D10565
:1014D30013E51370020514221231A8800312319010
:1014E300120F38121612129A11756A2075150175AA
:1014F300A6FF754A0112797A12790D127B2F121504
:10150300CAD5150975151E1215EE129A171216E093
:10151300E5791294D1E57EC333500274FF1294D15E
:10152300E5711215AF1294D1E5701294D1E57B24C5
:10153300ACFFE55F34091294D7EF1294D1E515207F
:02154300E03591
:10154500857D56E41294D1E52EC41294D7129539AF
:10155500129A1710021C205502809274401294F7BB
:1015650074451294F7744F1294F774461294F71257
:10157500953902122EE556121589C4FAE57D121524
:10158500892A80C0FBC41215962323CB1215962BEE
:1015950022540FFC24F650027C009015A5EC9322F2
:1015A50000000101010202030303FA2440400A245A
:1015B500804003EA3322D2E72274FF2220E703C3E7
:1015C500132224C022E53F701F7F7B7E0078AEE6A4
:1015D500128F05EE2404FE743A1290C2EE2404FE26
:1015E500E53E128EFF1298F822E53D1294EAE53E9B
:1015F5001294EAE53F1294EAE41294D1E41294D1EC
:10160500740A1294D174C01294D10295397440129F
:1016150094F774541294E5744E1294F7740012946E
:10162500D112169774101294EAE41294D11216BCD2
:10163500783D121C72E5121294EAE5111294EA74CF
:10164500011294D1901716121708756A101279D8DD
:10165500057F057F787F1294CA787B1294CA787DBE
:101665001294CA78771294CAE4FEFF78071294CAD6
:101675001294CAE5741294D1E5751294D1E41294CA
:05168500D1E573C33341
:10168A00500274FF1294D11294CA02953975C70395
:10169A0075C6FF75B901C217751D0085BC1C85BDCD
:1016AA001B85BE1A85BF19123AAAEE1294D1EF020F
:1016BA0094D1E5601294D11210FB128790E53A1288
:1016CA0094EAE53B1294EAE53C1294EAE53D129469
:1016DA00EAE53E0294EAE5751294D1E5741294D1D2
:1016EA00E5731294D1E5781294D1E5771294D1E595
:1016FA00761294D1E55E1294D1E57A0294D175A757
:10170A0000E493700122A31294F780F55843542DF4
:10171A00464C494748542000AF1F7E0478ADE61274
:10172A008EFF7E0C742C1290C27E0E18E6128EFF6B
:10173A007E1A78AEE6128EFF7E22743B1290C27E2B
:10174A0024E53E128EFF7E2FE540128F057E377408
:10175A003B1290C20E0EE541028EFF753200121046
:10176A00FB128790857946787A79641287A974641E
:10177A00123EA4121851756A20D26F1279D8537585
:10178A001F121888306F06C26F8E1E8F1FE57F608A
:10179A002BE54C24FFF54CE54D34FFF54D454C60E7
:1017AA000512792B80D5751D3C1279D853751F12F5
:1017BA00790D121888E57F6003D51DED1218E9909E
:1017CA001901129053AE1EAF1F1218E99018FA129F
:1017DA009053E546FD700B902E68305D11902E6493
:1017EA00800C047010902E64305D03902E607F3858
:0317FA00122E2C80
:1017FD00804BE4FFFC7E05305D047E027FB3123C1E
:10180D0030AC06AB07123AFA7F38C26FE51C6007A1
:10181D00D26F7E2C1290A3E51B206F026007D26F52
:10182D007E301290A3E51A206F026007D26F7E34CE
:10183D001290A3E5197E381290A3122E31E53224B1
:10184D00C850FA22E54075F03CA42541FFF54CE463
:10185D0035F0FEF54D7C007D10123C3D0F8F4BAFEA
:10186D004CAE4D7C007D3C123B107C00AD4B123CD0
:10187D003DEE4F70010F8F4C8E4D2278647973C2FF
:10188D00D112189FFF78677976D2D112189FFE0278
:10189D00997CC3E796FB0809E796FC0809E796FDD6
:1018AD00A2E792175003123DDE75135A30D10E7513
:1018BD001320B217AA47123B44AB04AC05E54660B2
:1018CD000B04600BAA46123B5BEB03FBEB03FBEB3C
:1018DD00543FFBE5132B2017029B9B22EE14143073
:1018ED00E701E4FEEF141430E701E4FF2205057073
:1018FD0088A8887005052020F82020753200129ADE
:10190D008B7E1E7F1C12997CDFFB12997C7E1E7FC5
:04191D001C12997C83
:10192100DEFB7E1D7F1D12997CDEFB7F007E217810
:10193100ADE6128EFF7E29742E1290C27E2D18E61E
:10194100128EFF7E35742E1290C27E3918E6128EE9
:10195100FF7F077E2174541290C27E25744F12902E
:10196100C27E2D78AEE6128EFF7E35743A1290C299
:101971007E39E53E128EFF78AE121C727F0E7E21FB
:10198100744C1290C27E2574411290C27E2DE512D4
:10199100128EFF7E35743A1290C27E39E511128E95
:1019A100FF7F157E2574441290C27E2DE540128F73
:1019B100057E35743A1290C27E39E541128EFF7F61
:1019C1001C7E2F857154128D527F217E01901C5FE8
:1019D10012496D7E0EAC77AB76128FC67E2B857960
:1019E1005F85787B1293137F287E01901C631249D7
:1019F1006D751D2B751E10E574121C037E25742F49
:101A01001290C2751D2D751E2BE575121C037F2FBB
:101A11007E02901C5712496DE5736003121A9E7F76
:101A2100367E02901C4F12496DE572121A9E121BEE
:101A31000B1210FB756A20AE4DAF4C7C007D40123D
:101A41003C3DBF00010F0FAC07AD07E4FED26F12A2
:101A510079D8127A24121AB4E57F602CE54C24FF60
:101A6100F54CE54D34FFF54D454C600512792B8061
:081A7100DE751D3C0E1279D850
:101A7900127A2412790D121AB9E57F6003D51DED8A
:101A89007F78128B767F767E0074301290C2E532B1
:101A990024C850FA227E21128C84128F0B7E2D903D
:101AA9001C67305D03901C6D02496DDD03AD040EAA
:101AB9007F78E55E20E72AE57A8549F0A4A9F0E573
:101AC9007A854AF0A429F9E435F0FAE55E8549F00A
:101AD900A429E435F02AFAE55E854AF0A42ACF9FC5
:101AE900FF12997C106F18C3EF9B50131BEF6B60AB
:101AF9000E8F018B0712997C1FEF6970F8AF01AB4C
:101B09000722901BC8305C03901BE1754A40754958
:101B190000AF76E577FE20E76B7005EF241050647F
:101B2900EF24A8EE34FD4011901BCD305C03901BCF
:101B3900E5754A1975499A8075EF2450EE34FB40D2
:101B490011901BD2305C03901BEA754A0C7549CD84
:101B5900805CEF24A0EE34F64011901BD5305C0375
:101B6900901BEF754A067549668043EF24F0EE3401
:101B7900F14013901BD8305C03901BF4754A04752F
:101B89004944802A8028EF2490EE34E84011901BC4
:101B9900DB305C03901BF9754A0275498F800F9001
:0B1BA9001BDE305C03901BFE754A0140
:101BB40075499A7F407E0012496D7F46128B767F6D
:101BC4005F028B763230305E003530305E00312279
:101BD40000322200332200352200382200464C37DE
:101BE40000464C313600464C333300464C36350003
:101BF400463130300046313630004632363000AEA1
:101C04001E75F064305C0375F03284C0F0F8700423
:101C1400EE2404FEE51D1290C2EE2404FEE86007E3
:101C24001290A3EE2404FED0E075F00A305C037534
:101C3400F00584A8F01290A3EE2404FE742C1290F4
:101C4400C20E0EE8305C01230290A35E25264053A9
:101C54004F47005E25264054415300414C540056E2
:101C640041520040225E2F2400404B545300E53E75
:101C74002541F51124C45003F511D3E63540F5127E
:101C840024E85002F51222C210129A8BD234127E2A
:101C9400B87F057E09901CB312493C7F157E0890DD
:101CA4001CE41290537F2B7E01901D4C02905341F3
:101CB4004952434F54454300532F4E0056312E3062
:101CC400362D30342D37004F4646214E4557404D72
:101CD400454E550020202040202020202020200098
:101CE400113007FE1FE001E101F80F00061B00F8A8
:101CF4000C00180E007C10007006003C2000E0066A
:101D0400003E4001E004001E8003C004001F0003E5
:101D1400C004000F00078000000F80078000001738
:101D2400800F00000027C00F00000043C00F001008
:101D34000083E00F00200301F00700C00F01F80347
:101D440083007F87FE01FC000E3E180000030000A4
:101D5400000018000003000000003800000000002C
:101D640000003000000000000000FC761F0E1C6024
:101D740030ECFCBC3F172DF0F978613866264F61D2
:101D84009A706070C60E1EE330E06060C60C1CC31F
:101D940060C0E0618C0C18C7C0C0C0E18C1C39C69F
:101DA40011C0C4C19C9931963180C8C1FF1E31E76E
:101DB400E180F0C0EE1C31C38180C2AFD2C075C0D7
:101DC4000075C70375C6FB852EBC8581BDD0BED00A
:101DD400BF123872C2AF74FE127EAB7F64129A19BE
:101DE400C2B480FC75C703E54875F004A42480F5EB
:101DF400C6C26E75B901E5BC047002D26E221232FD
:101E040024D269E5A62406500D3098F7C298E599C6
:101E1400B4E0F012325AC26922753400753703C235
:101E240028D229D22A75C703E54824E85003754807
:101E340000E54875F004A42480F5C67516077517E7
:101E440000C26E121E5C121E5C121E5C121E5C85A9
:101E54001758155875590022206E1D75B90105C60D
:021E6400AABC16
:101E6600ABBDACBEADBFEA121E7DEB121E7DEC1201
:101E76001E7DED121E7D22206E07F515B4FF03D2DE
:101E86006E22C0C7C0C612500275A704851683E528
:101E960017C4F8F58275B90105C6E5BCF0C582F828
:101EA6002406F92403C582E5BDF0E5BEF0E5BFF0E2
:101EB60075B90105C6E5BCF0E5BDF0E5BFB42F0375
:101EC60085BFBEE5BEF08516838982E4F075B9014B
:101ED60005C685BC1385BD14E4F0F08882E5BEF026
:101EE600E5BFF075B901E5BCF0E5BDF0E5BEF0E58E
:101EF600BFF0758306E51723541E24B0F582E5135B
:101F0600F0E514F075A700D0C6D0C70517221280D9
:101F160013C225C254C255127A6E754800121E1D90
:101F2600C229C22AC227C26AC268121F6CE4F537E8
:101F3600F52EF534F52F78A8F678AAF678BFF67858
:101F4600C2F6C236C252C222C223754601C215D299
:101F560021C219C226C23485705778B67401F608B4
:101F6600F608F608F622E4F542F541F54022121F7E
:0B1F7600141260DB121E02789F7680C0
:101F8100D210C211C212C213E4F54A78BAF608F6A9
:101F910078BC767878BD76051277EF75A60A12843B
:101FA100481222C6E5A624FA400312320420250B6A
:101FB100E535249C5007E59020E202806BE5322450
:101FC10010401978BEE6247D653270101297B47FF7
:101FD1000A7E181299AC1298F81225BB3098C5C226
:101FE10098E599B4E0BE12325A1225BB122278123A
:101FF10070DB127BD31225BB1260DB30121D101E69
:1020010010127896E5510404F57F24FE4003757F94
:10201100FFC277E54024F05002D255021F9C535471
:102021004F52494E472E2E0075A6FFC210301203A3
:1020310012203CC212752F000200FE123245127AA4
:1020410045129A8BE47E057F1E90201F12493C1297
:1020510098F8129A09D214D22012062C852BBC753D
:10206100B90575B902120622789D86BE75B9057546
:10207100B902127A4FD25512794F7F0012787CD271
:1020810020127A4FE56A600512790D80F7857A6230
:10209100D22012064585BEBC85BFBD856BBE856C51
:1020A100BF75B90575B90285BD6C85BC6B756A20B4
:1020B100127A45122104127A4F756A001279D8E515
:1020C1007064FE70397570FC854077854178851F95
:1020D100797818797A1287A91278F2D220129A1790
:1020E100127A4F756A101279D88554717F08781069
:0E20F10079721287AB85627C855E7D1278F273
:1020FF00C220C2142278107F0EE4F608DFFCF564CC
:10210F00F565F567F5687515FC751AC0751DC07511
:10211F006640756940754A0112797A30550302217C
:10212F00BD12790DE571B510004002F510E57EB5D1
:10213F0011004002F511E512207502E513C39579E0
:10214F005006207542857913D3E57A9514E5156409
:10215F0080FFE55E64809F400C857A14855E15854F
:10216F007B16855F17C2D17864797312219B7867CC
:10217F00797612219BD2D17818797312219B781B13
:10218F00797612219B808E85791280BCD3E79608D1
:10219F0009E7960809E66480FFE764809F20D10174
:1021AF00B3400AE7F61819E7F61819E7F622781878
:1021BF007964C2D11222197418123EA4AE1EAF1F39
:1021CF00781B7967D2D1122219C3E51F9FE51E9E96
:1021DF0050048E1E8F1F7EFF7FFFAC1EAD1F123C63
:1021EF003D7A04EF8AF0A4E5F0CE8AF0A42EFEE447
:1021FF0035F0BEFF011E60051460057EFF8E1F22A5
:0B220F00EE7E0020E7F77EFE80F3C3A8
:10221A00E697FB0809E697FC0809E697FD181819DE
:10222A001930E703123DDEC3EB33FBEC33FCED332D
:10223A00FDEB33EC33FBED33FC30D105AA47123BFF
:10224A005B0BBB00010C751E03751FFFEC24FC40E1
:10225A00048C1E8B1FE627FB0809E637FC0809E6F3
:10226A0037A2E713F618EC13F618EB13F62278BC2C
:10227A00E66048307345E57124F5403F16E624C40C
:10228A00403978BBE6255CF618E6355DF608C3E604
:10229A009560F618E69561F678BCE6701E78BBE69E
:1022AA00FF18E6FE7C007D3C123C0A75C70375C622
:1022BA00FE1277E58FBC8EBD1238722220125A3078
:1022CA00745110135778BDE53F75F00F84E5F0702F
:1022DA000806E624FA50027605E57124F65034160B
:1022EA00B600301232451260DB123245E4F534F59D
:0C22FA00372000253074EFD2207536121A
:10230600D22EE4F57EF55A127AA078BC7600122316
:10231600A0C21ED212C219121F6C121F5DC2202249
:10232600D26A120F25122332C26A80BB7F177E0043
:10233600908E3A12493C12063B85BC6285BD637598
:10234600A60AE5602562FBE5613563FC7F227E0413
:102356001290091298F8100008100110100220803F
:10236600DE1562E562B4FF0C156380080562E5625E
:1023760070020563E53524F550C575330180C0123A
:10238600063B1277E18562BC8563BD023872129AFC
:102396008B120EFF1223320201EFD2141223F6E63D
:1023A600F008DFFB857A621223EC7570FE783A79C5
:1023B600711287A91278F21223EC85627A855E7B08
:1023C60075C70375C6FE75B90185BC7E85BD7F756B
:1023D60070C01278F21223F6E0F608DFFB75A7004C
:1023E600757F01C2142274FF7870F608B880FB224C
:1023F60075A7049004F078707F10221210FB1287E4
:1024060090127BB99004EAECF09004EBEBF01231F9
:1024160090751F031216127F64129A19D51FF512B2
:102426001F14129A8B1298F8C25AC258C259756A6A
:102436002012797AD256123EA2754A0275430515C4
:102446004A753901C210D211D214D212127AA0756D
:10245600A6FFC221E54AB40202D221E535248C50FA
:01246600086D
:10246700E59020E2030224F9753609753200E54A42
:1024770020E00312955912797A1270DB20265F1239
:1024870060DB1543E5437020754303E54A30E018E8
:102497003057047405800F0404305605B4050780CF
:1024A70003B407027401F54A1225BBE54AB40402D6
:1024B7008003B40614AD3912797A202621DDF8E5B8
:1024C7003924DC400205398012753901E54A30E0CC
:1024D70006309803122514E53670CD0224551242B2
:1024E700A61260DE7536061225BBE53670F9C226E0
:1024F70080E9C211C212129A8B1298F8E4F535F5E9
:102507002FC22D7E06129A13C20202122EC298E51E
:102517003660241298A2B440F61298A2B44003126F
:1025270098A2B44912F5381298E0FC1298E0FBAD76
:10253700381298E06D600122C39004E9E0FF9B9098
:1025470004E8E0FE9C50048E048F038C148B137AEE
:1025570010123B3274202BF56A9004E7E03CF56BD0
:102567009004E6E03D540FF56C754A0112797AAE96
:1025770014AF137C0E7D10123C3D8F40AE04AF05A7
:102587007C007D3C123C3D8F418D429004EBE02561
:1025970013FF9004EAE03514FE7C0E7D10123C3DDB
:0C25A70078AEA607AE04AF057C007D3CBA
:1025B300123C3D8F3E8D3F2210001910010A10027C
:1025C3000A20780A20790A220226CC0226650226EE
:1025D300F7022686E53724FD5025602014601A3063
:1025E300101630741330121078BFE624FA4009062F
:1025F300753612D22E1263BC2202275C022796750F
:10260300340020112130741D201203D2132278A923
:10261300E670127602D277D226E536700575361249
:10262300D22E127A9522E54A20E008154AE54A702F
:10263300278022E543B40315205712154A154AE5AE
:102643004AB4FF09754A05305603754A03054AE53E
:102653004A24F95003754A01C256C2571291FA022D
:1026630098F8302909C229D22A7559008005302AE1
:102673000CD22912623B1262127534002220684088
:10268300202743D2221228D710790122E534243897
:102693004007753700753400227009E4C53770F5BB
:1026A300053780F11424FB400E24059026BE93F5D4
:1026B3003724FB40DD80DE740480F402030303044B
:1026C3001228B30228AAD26A22E53760271460567B
:1026D30014605F14601814601830101130120E303B
:1026E300370B78BFE6600616753612D22E22022803
:1026F300100227DED223122DAC10780122E53424F8
:01270300389D
:10270400400775460175340022700EE54624FE40EC
:10271400F1E54660ED154680EC04F54624FA50E5F3
:1027240075460580E0105B03D25B22100802D208D4
:1027340022205A08D25AC259D2588014205906D29B
:1027440059C258800B105804D2588004C259C25A36
:10275400E5346003D534DA222012047534002220D3
:102764002804D228801E126278055BE55B75F00BA5
:1027740084E5F0F55BE55A24F64009E55A955B508B
:1027840003755B0012627C1298F8E5346003D5345B
:10279400C722C252302804C22880253029030228C7
:1027A4007612623712624A102A240559C3E55895F5
:1027B400595005755900801BE558B4FF037559003D
:1027C40012625E1298F8E5346003D534C522755957
:1027D4000080EDD22A12623B80E920120475340095
:1027E40022302824126278155BE55B30E70C755BB8
:1027F4000AE55A24F64003855A5B12627C1298F863
:10280400E5346003D534D322D22880EEC252202886
:102814003E20293F12623712624A102A191559E5DF
:102824005930E715855859E558B4FF03755900D256
:102834002A12623B800E855859E558B4FF03755936
:102844000012625E1298F8E5346003D534BE22C2E9
:092854002880EE7F180548E548D4
:10285D0064187008F54830270375480A121DE830D2
:10286D006E05DFE875480A80237F181548E5483066
:10287D00E705754817800A64097006302703754807
:10288D0017121DE8306E05DFE275480A121E291277
:10289D00423CE532244C500512621280031261E86D
:1028AD007534000298F875A704758307E559C4F5CA
:1028BD0082E0E0F573E0F574E0F575E0F576E0F5AE
:1028CD0077E0F57875A70002423CE53424375031A6
:1028DD007005902917800A90292524FC4003902922
:1028ED001E7F3312290F0F12290F7F3C12290F0F54
:1028FD0012290F0F12290F7F357E0012493C1298B5
:10290D00F8227E301299ACDEFB22204241524F203C
:10291D000020575054532000404D41524B5340001E
:1060DB00129A8BE53724FD407978BEA6321297BB16
:1060EB00129607128C92128D34128F85128DB0126C
:1060FB0091FA128DCAE537600814602714603C8052
:10610B005CC2151261F9122EFE122E87E54824F699
:10611B005003122FDB122DD312969912431512999D
:10612B004D8024D2151261FFC26E122933122E3EFE
:10613B00129699124315129965800C1261FF128AFF
:10614B00451292B612993D126971126921128D9FF7
:10615B00800B600614601F0264071261E875A700CC
:10616B001292983022051228D7C222302305122D05
:10617B00ACC2230298F8120EFF12941F7F12128BDF
:10618B006430125075100075A7047583061242FD1A
:10619B00E51075F009A42415FFF5177E00E51260D4
:1061AB003575F06484E5F00F128EFF1F7E0EE5113E
:1061BB00128CEF7516231243C80510C3E55A9510C0
:1061CB004006E51024F550BF3012091262743028D6
:1061DB000312627C8087745D12910180CF120EFFD7
:1061EB0090634412628D202852202A4480653050DF
:1061FB00030267DB12913A201201223051061289F9
:10620B00CA0287B8028A26E4FEFFE54824F6400D51
:10621B0090633812496D7E16E5480290A390633E59
:10622B0012496D7E12E54824F7028F057D20800709
:0B623B007D3F3029027D3C7F00802861
:106246007D2D80167D2080127D3E800E7D3CE549A9
:1062560075F007A42406800A7D3FE55975F007A46A
:106266002409FF64027001FF7E1CED0290C27D2DA1
:1062760080067D2080027D3FE55B75F009A424162B
:10628600FF7E09ED0290C27E207F0012496D1262E8
:10629600127E007F0690632E129053E55804604CE0
:1062A60075100075A7047583071242FDE51075F099
:1062B60007A42409FFF5177E00E5121290C278069E
:1062C600EE2404FEE01290C2D8F6E51230E70A90FA
:1062D60062F37E2012496D800A7E20E5111262FC6F
:1062E60012442C0510C3E558951050B7224044457A
:1062F6004C455445440064B4602464B475F032845B
:10630600C0F01290A3CE2404CED0E075F00584C070
:10631600F01290A3CE2404CED0E0230290A3906383
:106326002A02496D2D2D2D000140FFFFFFE0FFFFE2
:10633600FFFF524F555445004C49535420004252DA
:106346004720214449535400787379AF1287A9E551
:10635600111263DE78731263B0AE04AD03E5110467
:106366001263DE78641263B0C3EB9DF518EC9EF5FC
:106376001E1244A1AC1CAB1B7A48123B32A91EA8C4
:1063860018123CD68B1F78AF79730287A91263DB8C
:1063960078641263B01244A1C237E51C7008E51B8D
:0463A600249B4002F2
:1063AA00D23775A700227F06E0F608DFFBE0FCE0A3
:1063BA00FB22127B9F1263DB401679067873E6F0A4
:1063CA0008D9FBECF0EBF0E55EF0E57AF075A70092
:1063DA002278BFE6F8601524F9401175A704758381
:1063EA0005E875F00AA424AAF582C322D322465FDF
:1063FA006E645000E51175F009A414FF22E4FFFE53
:10640A009065D812496D78BFE67003026168F5108D
:10641A00751101E478C0F608F61263FE0F7E007467
:10642A004C1290C27E04E5111290A3E5116510701A
:10643A000EE53F20E0407E0474201290C28037129D
:10644A00634E78C1E6251BF618E6351CF65002762F
:10645A00FF1263FE8F17AE1CAF1B75160C1243F5A5
:10646A0078C186071886067516211243F5AF177E7E
:10647A0035E51F128F0B0511C3E5109511509A12BD
:10648A0063938510111263FE8F17AE1CAF1B75162E
:10649A000C1243F578C1E6251BFF18E6351CFE50A1
:1064AA00027EFF7516211243F51263FE9063F8E52A
:0C64BA0010149360117E32128EBE1F1F62
:1064C600128B81EF240AFF128B817F417E00744A72
:1064D6001290C27E0474411290C21F7E0A74B812D2
:1064E6008EBE7517407E8C7F80C21712664C7E3238
:1064F600746C128EBE7F4A7E00744F1290C27E0468
:1065060074461290C21F7E0A74E3128EBE75174936
:106516007E007F20D21712664C7E32746A128EBEBF
:106526007F537E0074531290C27E0474411290C24F
:106536001F7E0A74FE128EBE7517527E0E7F10D213
:106546001712664C7E327467128EBE0261687F5BDC
:10655600128B64205B0C7F5F7E009065EB12496DA9
:10656600800A7F5F7E089066401290537F5E7E2889
:10657600742D1290FD7E2D740D128EB87E377446E2
:10658600128EB87F657E009065F612496D7F6C7E2F
:106596000090660312496D7F737E00906611124962
:1065A6006D7F7A7E0090661F12496D7F6A7E3390FA
:1065B60066301290537F727E327438128EB87E3CEB
:1065C60074001290DA7F7A7E3790662D12496D023A
:1065D60061684C45472021225E40212053225E40BF
:1065E60021225E24004041214032323530215E00B6
:1065F6002140202020225E2120202060004C3120D6
:1066060040323537212034352E38004C3220403187
:106616003435212032352E39004C3320403135387F
:10662600212032382E3200225E00070DFFF88D88B9
:10663600BAD88AD8B8D8BA88FFF80510FDC7FD863B
:10664600FC41FC41FD967C007D3C123C307C007D8B
:106656003C123C3DA805EFAF177E1E1290DA7E2352
:10666600743B1290FD7E25E8128EB23017087E1A12
:106676000F742D1290C222C25020092C30122920EC
:0F6686002826E558F46021D2508559101266B2CB
:106695001266F775A7049006DCE512F0E511F0E542
:1066A50017F0E510F0ECF0EBF075A7002275A704E4
:1066B5007583071242FD7813E0F608B819FA9006BB
:1066C500D07811E6F008B819FAE51CF516F0E51BC7
:1066D500F515F0758306E51023541E24B0F582E008
:1066E500F513E0F5149006DAE514F0E513F075A757
:1066F5000022120627E5BD75F005A4D2F785F01234
:10670500F511E4F51EF519F51CF51DC26F127A4554
:10671500128C48306F057519008054EB600B251DF0
:10672500F51DE4351CF51C0519051EE51E24C45090
:10673500DF128B5320D1388E1B8F1AE519FD24E209
:1067450050D4AE1CAF1D7C00123C308F19EF75F094
:10675500A7A4AEF0FFAC1BAD1A123C308F118E1200
:10676500C3EF94E8EE940340067512037511E790A4
:1067750006E2E519F01267B0AC16AB157AC8123B04
:1067850032E512C2E7F9A811123CD6ED7005EC24EA
:106795009E50057C807B0822C3E57A9513FFE55E54
:0A67A5009514FEC3EF9BFBEE9CFC75
:1067AF0022AE16AF157C00E519FD24FA501A123CE3
:1067BF00307C007D06123B107C007D05123C308F33
:1067CF0010EEF51724E950037517FF22201201224E
:1067DF0075A7049006D07811E0F608B819FA7F155E
:1067EF00128B647F32128B647F187E0078127519BA
:1067FF00071249C575A7049006D8E0F516E0F51500
:10680F00E0F514E0F513E0F512E0F511E0F517E00F
:10681F00F510E0FCE0FB75A700123ACC7F207E0557
:10682F00128F4C2017077E00746B1291017E1F741C
:10683F0063305C0274651291017F187E26AC14AB35
:10684F0013128FC690691D7F2B7E0012496DE517BD
:10685F00F46022AE17AF107C007D3C123C3DA805C2
:10686F00EF7F2A7E0C128EB87E16743B1290FD7E3F
:10687F0018E8128EB2E51233926DC313FEAF117C7E
:10688F00007D0A123C3DA805EF7F207E30128EB8A6
:10689F007E3A742C1291017E3CE81290DA7E292008
:1068AF006D080F74451290C280057467129101C371
:1068BF00E57A9513FFE55E9514FE92175003123D8E
:1068CF00C6AC16AB157AC8123B32A906A807123C04
:0168DF00D6E2
:1068E0007E037FE7ED700CEB2418EC34FC4004AE23
:1068F00004AF037C007D0A123C3DA805EF7F2A7E91
:1069000030128EB87E3A742C1291017E3CE81290BF
:10691000DA7E29746C301702742D029101455445BA
:106920000030504C75A7009006E0E0A3FCE0FBECC3
:10693000A2E79217402024FE50047F3B8022AE0441
:10694000AF037C007D14123C3D74542F2017029F2E
:106950009FFF7462800C123DD6EC24FE50E07F6DE8
:10696000743D7E001290C27E017D197C031269B6CF
:1069700022200A237E3E7D057C0B1269B6E579FD57
:1069800024C350027D3CED04C31304FD7F563075D3
:106990000712699F1FDDFA2212699F0FDDFA227E1E
:1069A0003C1299ACBF560312997C0E12997C0E12C0
:1069B000997C0E02997C7F3D12997CEF2DFFDCF8CB
:0169C00022B4
:10292D00D26E79B57700127A45E4F510F511F512EE
:10293D00F513F514F515F516F517C26F122AE020EB
:10294D006F1F122AE0206F19E51F30E51130E40EDC
:10295D001229A0306E0879B5E724F5500122D51063
:10296D00DBAE14AF157C00AD12123C0A8F55AE16BE
:10297D00AF177C00AD13123C30123E507E00E55572
:10298D0030E7011E2DFFE43E30E7027F00740A2F71
:10299D00F55622C235E51CAF1DBFFF050FD235F42C
:1029AD0004FABF003F752C00E518AF19BFFF050FE6
:1029BD00D262F404BF002D20E72A205B0123FF24FF
:1029CD00AA4021E51AAE1BBEFF050ED261F404BE6E
:1029DD0000128547F0A4E5F020E709205B0123FEF6
:1029ED0024AA5001227C567B1F305166302163C0D2
:1029FD0006C0078AF0E545A4AEF0FFE556205B0161
:102A0D001375F009A4ACF0FD123C3074FFBE00014B
:102A1D00EFFA24C050027A3FD007D006E552129843
:102A2D003D303504B2D5B2D1EA8CF0A430E70205C1
:102A3D00F0745625F020D10495F095F0FCEA8BF05A
:0A2A4D00A430E70205F0741F25F025
:102A570030D50495F095F0FBEC2F2062029F9FFF85
:102A670024884017EF24CB5012EB2E3061029E9E34
:102A7700FE24C04006306E0479B5072212997CE522
:102A87001E24FB50F60E12997CE51E24F650EC1E10
:102A97001F12997CE51E24F150E11E0F12997CE567
:102AA7001E24EC50D60F12997CE51E24E750CC1F4C
:102AB7001F0E0E12997CE51E24E250BF1E0F0F1247
:102AC700997CE51E24DD50B30E12997CE51E24D8AF
:102AD70050A91E1E1F1F02997C206F1912795812C8
:102AE7007841E4F5F7C2B2C2B2E5F7D2B2C22064C8
:102AF700C07003D26F22056D056D1278417D008D80
:102B0700F7C2B2C2B285F71F8DF7C2B2C3E5F79518
:102B170073F5188DF7C2B2C2B2E5F79574F5198D42
:102B2700F7C2B2C2B2E5F78DF7C2B2C3E5F7957641
:102B3700F51A8DF7C2B2C2B2E5F79577F51B8DF797
:102B4700C2B2C2B2E5F78DF7C2B2C2B2E5F7F51E5F
:102B57008DF7C2B2C3E5F7957AF51C8DF7C2B2C2FD
:092B6700B2E5F78DF7C2B2C2B26B
:102B7000E5F7D2B2C220543F30E50244C0955EF57D
:102B80001D156D156DE51024784001227E00AF55AE
:102B9000EF30E7011E0512E51FA2E592D5400EE5D4
:102BA00015951EF515E5149400F514800BE5152513
:102BB0001EF515E43514F5147800E51E600620D5E1
:102BC0000318F404C39FF5F0E89E30E701220513D3
:102BD000E5F0A42517F517E5F03516F5162274541F
:102BE0002F2062029F9FFF741D2E3061029E9EFE69
:102BF0002279B4203245201D42EFB506009260AC28
:102C000006AB074004AC07AB06902C3CEC230493C6
:102C10008BF0A4A9F0EC23938BF0A429F9902C9CC1
:102C200093C9902D9CE52C9313E95001F4902DA4A9
:102C3000F9E52C932975F0B484A9F022FFFFFFFF7A
:102C40007FFF55553FFF33332AAA24921FFF1C7183
:102C500019991745155513B1124911110FFF0F0F8F
:102C60000E380D790CCC0C300BA20B210AAA0A3DB0
:102C700009D8097B092408D30888084207FF07C13F
:102C800007870750071C06EB06BC06900666063E43
:102C9000061805F405D105B0059005720000000086
:102CA000000101010101010101010202020202020F
:102CB00002020203030303030303030304040404E3
:102CC00004040404040505050505050505050606B7
:102CD000060606060606060607070707070707078C
:102CE0000708080808080808080808090909090960
:102CF00009090909090A0A0A0A0A0A0A0A0A0A0B38
:102D00000B0B0B0B0B0B0B0B0B0C0C0C0C0C0C0C0C
:102D10000C0C0C0C0D0D0D0D0D0D0D0D0D0D0D0EE6
:102D20000E0E0E0E0E0E0E0E0E0E0F0F0F0F0F0FBD
:102D30000F0F0F0F0F0F1010101010101010101099
:102D40001010101111111111111111111111111176
:102D50001212121212121212121212121213131350
:102D6000131313131313131313131313141414142F
:102D7000141414141414141414141415151515150E
:102D800015151515151515151515151616161616EE
:102D900016161616161616161616161600FFFF002D
:102DA000FF0000FF002EB5875B2D5A88E5342437DD
:102DB0004001227F357E2B7D0F600C7D1E14600745
:102DC0007D3C1460027D78ED305D02C313128E6489
:102DD0000298F8E546604A14603C14602E146020A6
:062DE000146012902E7C2D
:102DE600205D41902E807F367E34129053803C9039
:102DF6002E7C305D03902E78802A902E78305D03ED
:102E0600902E74801F902E74305D03902E70801467
:102E1600902E70305D03902E6C8009902E68305D88
:102E260003902E647F367E3312496D1F7E3C7422DA
:102E3600305D027466029101305D08902E54305B5D
:102E4600E38006902E5C205BDB902E5880D6302CDB
:102E56003500312C3000322C3000302C3600312C2D
:102E66003200322C3500332C3800372C35004031F7
:102E7600350040333000403630000508B28D8DB540
:102E8600BAE558B4FF0122780075A70475830712C6
:102E96002F5588198A1A8E1E8F1F30D14EE546701F
:102EA60034E54824F6402EE865597029120631E5C6
:102EB600BD602275F005A475F00984FD122BDEEEC7
:102EC6002402F8EF2402F97A00EA12983D1299DCFE
:102ED6000A0ABAB4F4AE1EAF1F122BDE1EE51A1292
:102EE60090C2EE2404FEE5121290C2A81908C3E5AA
:102EF6005898509575A70022780075A70475830623
:102F0600122F5530D139122BDEE54624FE500A0E1B
:102F16000F902F501290538026EA7007745D12901E
:102F2600BE801C75F06484ADF0700FED75F00A84F8
:102F36007008E5F00E1290A380051EED128EFF08B4
:102F4600C3E55A9850B475A70022030340A040D2A7
:072F5600D1E8C4F582E0FAA6
:102F5D007973122FAB30D143AF06752C00EDBFFF47
:102F6D0007F40460360FD262BF00301230D1402B0F
:102F7D007976122FAB30D123E5822403F582E0F56B
:102F8D0012EEA2E713FEED13BEFF07F404600C0E64
:102F9D00D261BE00061230EE400122C2D122C3E042
:102FAD009709FDE09709FEE097600904700AEE307D
:102FBD00E7068007EE30E703C2D122E546600E1426
:102FCD00600BF9EDCEA2E713CE13D9F8FD227C00EC
:102FDD007B44E54660207C007BCC1460197C017B32
:102FED00981460127C037B3014600B7C067B60149C
:102FFD0060047C0C7BC08C148B157AE9123B32A8D3
:10300D0047123CD48C168B1775C70075C604751006
:10301D00DF75B901E5BC20E76FF51385BD1205C657
:10302D0005C675B901752C00C3E5BE9573FBE5BFEB
:10303D009574FC05C675B901E5BC9575FD5005D2B5
:10304D0062123DDEC3E5159BE5149CE49D40338C77
:0E305D00198B18C3E5BD9576FBE5BE9577FC93
:10306B00E5BF9578FD5005D261123DDEC3E5179B98
:10307B00E5169CE49D400D8C1B8B1A1230A6E53295
:10308B002428401305C6E5C68006E5C62404F5C60C
:10309B00700205C7D510012202301EAE19AD1812F1
:1030AB002FC8ED1230D1AE1BAD1A122FC8EE13ED97
:1030BB00131230EE122BDE1EE5131290C2EE240417
:1030CB00FEE5120290C275F0067FFDA946B9000518
:1030DB0075F0027FFF84C5F02F500205F0C5F0FF9D
:1030EB0024DE228547F0A430E70205F0E5F0A9467F
:1030FB00B9000280050475F00384FE24E022E53755
:10310B007002D27E64027002C27EE53724FD79B56F
:10311B00E76005640B600C22D27C20081E401C105B
:10312B007D1022D27D2008134011107C01227537AF
:10313B000122753700207E0375370222123150E5CC
:10314B00BC14601822120631E5BC60101460189094
:10315B0031EA75F9FF75FBFFC253804475BC0090D3
:10316B0031D212318880219031DE1231888031E5E5
:10317B00BC640260049031F6229031FD22D253E4FC
:10318B00F5F9F5FB22123188759E85759D2D759885
:01319B0052E1
:10319C0022123188759E84759D2D80F112318875AF
:1031AC009E83759D0980E6123188759E82759D09F6
:1031BC0080DB12319075F9FFC25322123188759E53
:1031CC0081759D1180C7574952452040392E3622B2
:1031DC00200057495245204035372E36220049529F
:1031EC0044414035372E3622200020574952452085
:1031FC00002049524441200012063675BCF605BD2C
:10320C0075BE00123872D2A47F64129A19C2A4122D
:10321C00956B1298F8129A0975A6FFC2141231BE5A
:10322C0074C01294E574A31294F7748F1294F7E59A
:10323C00381294F774CA0294F7C274C273E4FDF5A1
:10324C0071F5701298A77003DDF922B4E0F5F5382A
:10325C00753200C274C27375A7049004B41298A29C
:10326C00F0A2E29274A2E192731298A2C2D112332C
:10327C00DC20690330740B8D758E748F73E514C468
:10328C00F57D12345C1233DC20690330740C8D78BC
:10329C008E778F76E514257DF57D12345CD2D112B4
:1032AC0033DCEEF0F55DEFF0F55C1298A27D0A12BE
:1032BC0034498F71EE60037571FF7C007D05123C03
:1032CC003D8F517D141234498F701298A2F054071F
:1032DC00C52E54F8252EF52E1298A2E5386002D290
:1032EC001E1298A2B4E1FA1298A2F01298A2F0F56C
:1032FC003A1298A2F0F53B1298A2F0F53C1298A263
:10330C00F0F53D1298A2F0F53E1298A2F0F53F129E
:09331C0098A2B4E2FA1298A2F0A2
:103325007E0C1298A2F07F051298A2DFFBDEF31245
:1033350098A2B4E3FA7F041298A2DFFB1234491273
:1033450098A2B4EAFAE561F0E560F0E55EF0E57AA9
:10335500F0E579F0E52EF0E55FF0E57BF0E57EF050
:10336500E4F0F0F020740C9004BFE4F571F570F012
:10337500F0F0F075A70078ABA63A08A63B08A63C86
:10338500120631E5BF253D240C75F0188478AEA6EC
:10339500F0186005640260182216E670121816E629
:1033A5007004760C181678ACE69033CF9308F622A5
:1033B5000618E6089033CF930466700D760118065B
:1033C500E6640D70047601180622001F1C1F1E1FDF
:1033D5001E1F1F1E1F1E1F1298A2FC1298A2FD126F
:1033E50098A2FE1298A2FFECA2E692E7921713FCB0
:1033F500ED92E713FDEE92E713FEEF92E73017012A
:10340500F4F513ECA2E713FCED92E713FDEE92E75A
:10341500301701F4F512ECA2E713301701F4F5109B
:03342500ED92E73E
:10342800301701F4F511123D6720D10E8C1C8D1D4B
:103438008E1E8F1F123DA7123D67301703123DB82D
:10344800221298A2C313FEF01298A292E7FFF07C12
:1034580000023C3DAC1CAD1DAE1EAF1F3017031261
:103468003DB8ECF0EDF0EEF0EFF022123479020204
:1034780090129A8B7F517E059034A612493C12987F
:10348800F8123190129A09C2021298A210020EB4D0
:103498000DF7129555129A0912955180EC22535442
:1034A8004152545043392E36004C4F4144494E47FF
:1034B8002E00D2201234C4C220020290121E021220
:1034C8009A8B7F5A7E059034B112493C1298F8D2F3
:1034D80014C255121F6C789F76800876001277EF19
:1034E8001223EC7570FE853A71853B72853C7385B5
:1034F8003D74853E75853F761278F21223EC75701F
:10350800C0757B03757A54E4F57FF57E1278F27501
:103518001421751348755F01757B00757504757402
:103528005275780175776CE4F57DF57E757F0190AD
:10353800D63485836E85826DC26F1235A2851C1DB7
:1035480075A6FF3055067554B502203F1235A2E521
:1035580072A2E59275A2E79277D274D273E51275DA
:10356800F008A4AEF0FF207503123DC6128723129F
:103578008767123625E51C251D13F571851C1D78F6
:10358800BF7600127800127896757F027F5A7E35D2
:08359800E541128E471298F87C
:1035A00080A6856E83856D82C25578731236067843
:1035B00076123606E493F570B4B402D255A3E493C0
:1035C000F51CA3E493F512A3206F0FA97BE493F5F8
:1035D0007BC399502A20E702055FA385836E85820D
:1035E0006D106F16D26FE5822405F582E43583F500
:1035F00083E493F52654F0F57222E526C480F63074
:10360000E7D8155F80D48601E493F6A308C39950E8
:103610000A20E70606B6000208062230E70616B6BC
:10362000FF0218162230750DE5132579F513E435E0
:1036300014F514800DC3E5139579F513E514940082
:10364000F514AE14AF137C007D0A123C3D8E5E8FE4
:103650007A22120636E5BE04600A9036657E057F42
:103660006312493C222E0012063675B905020290FB
:103670002275A6FF120636E5BE0460439036C07E72
:10368000007F5A12496D9036D27E147F6112496DC7
:103690009036D97E087F6812496D7F707E00E5BC48
:1036A000128EA57E0FE5BD128EA57E1EE5BE128E82
:1036B000A57E2DE5BF128EA57E3C74061290DA22FF
:1036C0004552524F52434F4445404D41494C544F4F
:1036D0003B004F46464943450061414952434F54E0
:0E36E00045432E415400120640E5BC046073C1
:1036EE007F5D7E08901CBC12493C7E20E5BC129189
:1036FE00017E26E5BD1291017E2CE5BE1291017E62
:10370E0032E5BF1291010298F87E057F6C90375A10
:10371E0012493C1298F8D26F7E2975135012374910
:10372E0075134812374975135012374975134B12DA
:10373E003749306F03123761020290785F1255DA03
:10374E00E865136002C26FEE2406FE224643545211
:10375E00593A00C210C21175B90675C70375C6FC79
:10376E001277E175BC2812387275C6FA75BC0275EF
:10377E00BD1475BE0075BF0C12387275C6F812777F
:10378E00E175BC3275BD0F12387212387D75333249
:10379E00120EFF75C70375C6FC75B901A8BC75A6D8
:1037AE00FF7F4B7E009038F812493CE8128EBE889F
:1037BE00177F0F7E121292BAA8171298F8100008EF
:1037CE0010010710021880D618180853003F75C74D
:1037DE000375C6FC1277E588BC12387280C075C7B7
:1037EE000375C6FF74301277E675BC331238721249
:1037FE0036EE120F0E75130380097E20A8BC1255EB
:10380E00FF88BC7F747E36E513141290A3C26E7FC0
:10381E005D7E26A8BD1255FF88BD7E2CA8BE125512
:10382E00FF88BE7E32A8BF1255FF88BF306E03756B
:10383E001303D513C575C70375C6FF12387212323E
:10384E00241277C81234C475C6F71277E175BE40DC
:10385E0075BF0312387275C6F91277E175BC0E7515
:04386E00BD4C8000CD
:10387200D22075B90575B902C22022123224129AD9
:103882008B7F007E0B9038EB12493C120F1E7D009D
:103892001298A77004DDF9802EB4E2F41298A2F512
:1038A2001375120C7511061298A2D511FA6015F44F
:1038B2002460FFE51275F005A4FE12997C0FC3EF98
:1038C200944740F6D512DD7F287E0E9038F31249D8
:1038D2003CE513128E4D7F32128B647F46128B644D
:1038E2001298F8300295C202225345525649434576
:1038F200005341543A00434F4E545241535400D264
:1039020014129A8BE4F56CF56BF56AC26FE4FEFF54
:10391200E56C128E647E14E56B128E647E28E56A75
:10392200128E64751E00751F041279D8206F421220
:10393200790DE53524B4500C127928E5352464500C
:10394200031279287F0A7870E608AE1E128F0BEFF9
:103952002407FFB880F2E51E2410F51ED51FCA12F7
:1039620098F875A6FF1000201001A010020280F244
:103972002212793BE53524B450CA127955E5352433
:103982006450C112795580BCD26F8081D214129AD0
:103992008B75C70375C6F0E4FEFFE5C7128E647E21
:1039A20014E5C6128E64751F107F0A75B9017E0078
:1039B200E5BC128F0B7E10E5BD128F0B7E20E5BE9B
:1039C200128F0B7E30E5BF128F0B05C6EF2407FF67
:0539D200D51FD8E5C679
:1039D70024F0F5C61298F875A6FF10001710010518
:1039E70010022080F2E5C62410F5C670A505C7535E
:1039F700C703809EC3E5C69410F5C6E5C79400F5D6
:103A0700C780EC22E4F5C7F5C675B90505C6E5C656
:103A170064E06008E5C670F105C780EDE5C764039B
:103A270070E7123A2F024E58E4F5C7F5C675BC2663
:103A370075BD4E75BE4575BF5712387205C675BC44
:103A47005775BD5075BE5475BF5F12387205C6E411
:103A5700123A5A1277E612387205C6227F5F7E0D38
:103A6700E56C128F0B7E1EE56B128F0B7E2FE56ABE
:103A7700028F0B7F657E1EE54B128F0B7E2FE54C69
:103A8700128F0B7F6B7E1EE54D128F0B7E2FE54E3F
:103A9700128F0B7F717E1EE54F128F0B7E2FE55025
:033AA700028F0B80
:10D6340069FC362E06FD69FC372F071169FD383069
:10D6440007FD69FD3931061169FE383107FD68FEB1
:10D654003732091168FF373008FD68FF372D07118D
:10D664006800362909FE680036290C116801372B39
:10D674000CFF6801372F0A116802383009FF68026D
:10D68400372E08116803372C0AFE6803372E081159
:10D694006704373208FE67043633091167053535E8
:10D6A40005FF6705353303116706362F02FF67064A
:10D6B400362B05116707362B07FF6707352F051132
:10D6C4006708353104FF6708332E051167093128CF
:10D6D4000700670931250A11670A35240B01670A17
:10D6E4003A240A11660A3C210801660B3D1E0B11FF
:10D6F400660B3D1E0C00660B3D200A11660C3B2197
:10D704000CFF660C39220E11660C37231100660DCE
:10D7140036240D11660D34260F01660E32261111C2
:10D72400660E32251401660F35251311660F37274F
:10D7340016016610392918116610392B1502651166
:10D74400392D11116511372E0C026512332F081172
:10D754006512312F07026513302C0A1165132D2928
:10D764000E0265132A271011651429270E02651469
:10D774002C290C1165153129080365153726071165
:10D784006515321F09036516411B09116516411CF5
:10D7940008036416461F081164164D210504641617
:10D7A4005922031164166425040563156A240711BC
:10D7B40063156D23090663156C230D1163156C2520
:10D7C400130762146E2B151162146E2F1406621364
:10D7D4006E30161162136E30150761136F3112111A
:10D7E40061126F350F0761126F380D116011723AB3
:10D7F4000A086011763F0611601079420209600F31
:10D804007A3A0533600F7832040A5F0F742C0133BF
:10D814005F0E722B030A5F0E732E08115F0E7430B5
:10D82400050C5F0D722C02135E0D6C2B010C5E0D4A
:10D83400622C05315E0D5F2B030D5D0D5E290833EF
:10D844005D0D5F23030B5D0D5F1B01335D0D5A16E8
:10D85400020A5D0D521B00115C0D4D26000C5C0E7E
:10D86400462802335C0E3926040C5C0F2C2B08333B
:10D874005C0F23320C0F5D0F172E0A335D0F0C2E35
:10D8840009105D0F043507335E0FB23C080F5F0FBC
:10D89400AB4209335F0EA43E070F5F0EA2430B3366
:10D8A400600EA746120B600D9F490C73610C9C49D6
:10D8B4000F0C610B97460973610B8B440A0C610AC8
:10D8C4008B420B336109843A080C6108823A0433B1
:10D8D40061087934030C60086F2F063360086228EE
:10D8E400050C6008572505336008511F040D5F08B7
:10D8F4004E1B05335F08491B090D5F094120103792
:10D904005F0938270D0D5F0A302F06335F0B2B326A
:10D91400070F5F0B282F0A335F0B262E0E0E600CA9
:10D9240023361137600D1F3F160F600D1841127713
:10D93400610D0F320A13610D042B0633610D022EA3
:10D94400040E620D043A0231620E0343050D630DA9
:10D95400B1470113630DA94A000B640CA14D0511D5
:10D96400640C9B44070E650B99490911650A944799
:10D97400090D65098E49021365088848060D650876
:10D9840081400E336407793B130F6407722F1877B5
:10D9940064076D231A106407692911776407651CED
:0DD9A400080F63075D180B33630751190D61
:10D9B1000D630746220E336308402B110F630838AD
:10D9C100291837630932271B0D6309312B1477623C
:10D9D1000A372C0F0A620A3C280973620A441E0B9B
:10D9E1000C620A48150E33620B46190C0A620B478A
:10D9F100260D33610B4C280C0B610B54251037613C
:10DA01000B5E24170C600B63291A77600A663614C3
:10DA11000A600A68390B735F0A6C2C100A5F09727D
:10DA21002015775F097422120A5F0873300F775F40
:10DA3100087639140A5F077D3816775F0785370F37
:10DA4100095F068D3B0D735F058B4410075F048BE7
:10DA5100490C735F048E3F0C075F03863604335F06
:10DA61000394280708600299300E1160029E400558
:10DA7100076102A34A0C336101AA4810086201B18F
:10DA810042127762020131150A6202062B13776393
:10DA9100020830110C63020B361277630310331145
:10DAA1000C6403182B147764032223110A640426DF
:10DAB10023107764042226110A64051C2715776454
:10DAC100051D251508640521271277640628270FEF
:10DAD1000764062F1D11776406350F140764063E8F
:10DAE1000A19776406401216086407431B1177630D
:10DAF100074A22120663075228127763075A27132F
:10DB01000662075E231477620661201107620664CC
:10DB11001E0E7362066A1E0E0762067421103762BA
:10DB2100057828130661057A2F157761047A332069
:10DB31000661047A301B7761037A281B0761037F32
:10DB410023187761028429160661028832177761EA
:10DB5100018D371305610193340C7362009A2E090C
:10DB61000562009D2E043362009D370C0663FFA001
:10DB710040103763FFA844140564FFAF4612776471
:10DB8100FF014511056500043F12776500053E1050
:10DB9100076600073F117766000B430D0767011009
:10DBA1003D117367011539120767021A321277673F
:10DBB100021A2C12076702192C107768031B2E0F0B
:10DBC1000668031F2C117768042729100468042EA6
:10DBD1002A0F776705322F130467053330127767F1
:10DBE10006362D140567063B291677670643231B66
:10DBF100046706471E16776607491E150366074C1C
:10DC01001B157766074C22170466075222147765A5
:10DC1100075B26150265066229157765066D2917CA
:10DC21000165067529137765057D281A0265058248
:10DC310028187765047F1F160265048F2A117765FE
:10DC410003953211006602993D157766029C401CCE
:10DC5100FF6602A13E1F776701A43F1CFF6701A772
:10DC61004314776801AB4710FF6901B1490F776928
:10DC710001024911026A0207490D736A020B480C3D
:10DC8100056B030F480B336B03144A0D026B041928
:10DC91004914376B051F491CFE6C06224824776C1A
:10DCA10006233F21FC6C07203023776C07212721B5
:10DCB100FC6C07262420776C08292812FC6C0828A4
:10DCC1002C0F776C0927230CFF6C09251802316C86
:10DCD10009350F05FC6C094C1401116C09561D0125
:10DCE100FC6B095F2003136B086B2108FB6B087445
:10DCF1002509336B08772507FC6B0778210D336BFA
:10DD0100077A1E0AFB6B077F220C336B06832E0AF0
:10DD1100FA6B05853C09336B0489410EF96B048C60
:0DDD21003E10376B038D3C0FFA6B038D40F5
:10DD2E0013776B02904112FA6C01934110776C01DC
:10DD3E00984410F86C009B471A776D009F461EF8AA
:10DD4E006DFFA24519776EFFA14019F86EFFA64030
:10DD5E0014776FFEAA4417FA6FFEAF4A127770FE61
:10DD6E00B34D18FA70FF024B1B7771FF054718FD74
:10DD7E0071FF0942177772000E4012FD7200163DB8
:10DD8E000C7372011B3510FA7201232E1577720275
:10DD9E0029321AF872032C371D7772032F3014F8BC
:10DDAE00720336210F77710346190DF87103502057
:10DDBE000B33710353290EF87003572B143770036E
:10DDCE00612712F870036F2911777002793017F7F7
:10DDDE007001803722777001843D1FF67000883FF6
:10DDEE00197770FF8D3F11F670FF933D0C7371FE26
:10DDFE00973D0EF571FE9B3E0C3372FD9F4310F660
:10DE0E0072FDA448127773FDAB4C13F573FDB14F41
:10DE1E00167774FD034F14F775FE074C127775FED7
:10DE2E000A4510F975FE0E400F7776FF124111F874
:10DE3E0076001745167776001C4614F676012142B9
:10DE4E0017777602263D17F3760229382177760367
:10DE5E002A3315F276032B3009737604302A07F035
:10DE6E00760439220A337604472110F075045125C1
:10DE7E0012777504552416F1750459210F77750420
:10DE8E005F2111F0740463231477740468240EF276
:10DE9E00740370230933740379270AEF74028030F8
:10DEAE000B33740185360DEF74018B391337740003
:10DEBE00903D1BF075FF94441E7775FF984823EF35
:10DECE0075FE9B46207776FE9F4221F076FEA13F9F
:10DEDE00177777FDA44313EF77FDA747157778FDE6
:10DEEE00AA4915EF78FDAD4C157779FDB04D19EEB9
:10DEFE007AFDB34D1C777AFD024E19F07BFD054F6E
:10DF0E001B777BFE094F24F37CFE0D531D777CFFA0
:10DF1E00114619F37CFF173F12777C001F3810EF64
:10DF2E007C00263613777C012B3115ED7C012F2BCF
:10DF3E0015777C02332513ED7C02392214777C028F
:10DF4E00402110EE7C0249210B737B02531F0FEB15
:10DF5E007B02601E15777B026A2214EA7B0174280D
:10DF6E0019777B017B2D1AEA7B00833122777B00A8
:10DF7E008A3320EB7BFF91371A777BFE953C1FEAA5
:10DF8E007CFE983C26777CFEA74621EC7CFD9939D9
:10DF9E0023777CFC9A3B1FEA7DFC9A3F1C777DFB26
:10DFAE009A401EE87DFB9B3F20777EFA9B3F1FE643
:10DFBE007EFA9C431A777EF99E4717E57FF8A04AB2
:10DFCE000E737FF8A34A0AEA80F8A548073380F853
:10DFDE00A94402EA81F8AE46041182F8B24C00E779
:10DFEE0082F80351021183F8085304EA83F90E4DA7
:10DFFE00061183F914430CEC84FA1A400E1184FBBB
:10E00E00203F0AE884FC2540061384FC2B4008E6DA
:10E01E0084FD3039073383FD36300EE483FE3C2B0E
:10E02E00193783FE402A1EE783FE3D25187783FEAF
:10E03E00371B16E783FF3114137783FF35170FE471
:10E04E0083FF3E220D738200412C15E58200432C86
:10E05E001A77820046251BE782004C201577810037
:10E06E00552116E581005E2510778100682718E49A
:10E07E0081FF72291E7780FF7A2E22E580FE7E3088
:10E08E00277780FE812B22E680FD85251C7780FD7B
:0DE09E00882618E281FC8A2F187781FC8DFE
:10E0AB003821E181FB903F287781FA924025E0816E
:10E0BB00FA943D237782F9973C18E082F99A3F1541
:10E0CB007782F89E4412E083F8A347107783F8A772
:10E0DB004A0CDF84F8AA4D133785F7AC5214E2854E
:10E0EB00F7AF56107786F7B2580DE087F802560255
:10E0FB003387F8055002E388F8094C051188F90CB1
:10E10B004E02E489F91052011189FA155004DF8986
:10E11B00FB1D45041389FB233304DE89FB292306EE
:10E12B003389FC2B1F05DE89FC2F23093389FD3333
:10E13B00280ADC89FD3B23103788FD471E0EDD883E
:10E14B00FD511E0E3388FD53200CDD88FD54210B31
:10E15B003387FD57200DDD87FD5C20093387FD5D7F
:10E16B002403DE87FD5B29013386FD592C04DE86F3
:10E17B00FD5D2C093385FD622F0CDC85FD652D0BB8
:10E18B003385FC672908DF85FC6722093385FC6B27
:10E19B00210CDD84FC72280A3384FB783005DD8486
:10E1AB00FA7C37073384FA7E390ADC84F9813B0623
:10E1BB003384F8843F05DB84F8873F023384F78A86
:10E1CB003C04DB84F78D390A3384F6903908D98502
:10E1DB00F5923F113785F595430FD985F498440A8D
:10E1EB007386F49B440AD986F39C440C3386F39CC8
:10E1FB004507DA87F29C47063387F19E4C0AD9888C
:10E20B00F1A251103788F1A65516D989F0A7571FDF
:10E21B00778AF0A9541BDA8AF0AA4D12778BF0ACEF
:10E22B00460DDB8BF0AC4906338CEFAB4D05DB8C2D
:10E23B00EFA95002318DEEA85209E28DEEA7530ED5
:10E24B00118EEEA75316E58EEDA44A20118FEDA08B
:10E25B004423E28FEC9C4821118FEB9A4A22E090E9
:10E26B00EB95411D1190EA8E391DDF90EA8936211D
:10E27B001190E9873223E590E9852C2C118FE87DED
:10E28B002A26E08FE8762124118FE8662122E08F81
:10E29B00E856221F118EE947201DE08EE939211621
:10E2AB00118EE9302518E28EEA2D2917118EEB30ED
:10E2BB003213E18EEB333711118EEC373C10E18EBC
:10E2CB00ED393E07138DED3B4203DD8DEE3B3E09F1
:10E2DB00338DEE3B310DDE8DEE392812378DEF3855
:10E2EB002319DC8DEF382A18778DF0372A12DC8D45
:10E2FB00F0382214778DF0361B0EDC8DF1361B0CAB
:10E30B00338CF1371F0DDB8CF136250E378CF23445
:10E31B00270CDC8CF22A270D338DF31F2A0CDC8D96
:10E32B00F3173409338DF4143A08E48EF4123A0CD3
:10E33B00338EF4103D11EA8FF50E411A778FF50CE1
:10E34B004917EA90F50A50157790F5054F13E791A9
:10E35B00F5B24F107792F5AD5408E492F4AB5A0135
:10E36B003393F4AB5C05E893F4A9500A3394F3A40C
:10E37B00450CE094F3A041093394F29A3A05E295E7
:10E38B00F29734043395F1913208DC95F19E310DFF
:10E39B003395F08A320CDA95F0872D0B3395EF809D
:10E3AB00250EDE94EF73220C3394EF6C2412DD9464
:10E3BB00EF6928157794EE6B2812DF93EE69280E20
:10E3CB007393EE64270DDF93EE5C260B3392EE57BF
:10E3DB00270EDB92EE5828123792EE5E2610DB9258
:10E3EB00EE64240D7391EE6C2108D991ED72230428
:10E3FB003391ED782904D991EC7C320A3391EB7F80
:10E40B003A08D891EB833D093391EA883C0CD791BC
:0DE41B00E98D3B103791E9903E12D792E851
:10E428009143137792E794420ED792E7993E0733C8
:10E4380093E7A03901D993E7A63B0A1194E6A83FD0
:10E448000CD794E6AB490E1195E6AE4F07D695E684
:10E45800004D011396E6034601D996E6033E0811DE
:10E4680097E7043D0ED997E70740151198E70C4345
:10E4780012DA98E812460F1198E918490CDA98E967
:10E488001D44081198EA243D05D898EB293A031150
:10E4980098EB2C3707D898EC2D38093398ED2E3D9A
:10E4A8000ADC98ED2E3E0A3398EE2D3F0BDB98EFF1
:10E4B8002C420C3398F02B430ED998F02B3D113792
:10E4C80098F12D3710D898F130340D7398F2343311
:10E4D8000FD698F237330F7798F339331CD597F363
:10E4E8003C32167797F43E2F11D797F440280973DA
:10E4F80097F4422109D797F4461F0AB396F44B21A3
:10E5080008D796F45325083396F45C2505D796F476
:10E518006723023395F4722503D695F3782B0231DD
:10E5280095F37B3102D695F27E31063395F1832F30
:10E5380004D695F18A2F023395F0913201D596F0E1
:10E548009638061196EF9A3F02D497EF9D4502132D
:10E5580097EE9F4704D497EEA247073398EEA64458
:10E5680008D398EEAA430B3399EEAD440CD499EE38
:10E57800B1400D339AEE013F11D39AEE054512775B
:10E588009BEE064A15D59BEE064712779CEF05428F
:10E5980012D79CEF063E0F779DEF084111D39DEFF0
:10E5A800094619779EF00B4718D39EF00D431C7748
:10E5B8009FF10F4015D69FF1114113779FF2134633
:10E5C8000ED9A0F2174A0B33A0F31C4A08D4A0F4C2
:10E5D80023420333A0F42A3305D3A0F531270711CA
:10E5E800A0F5382300D29FF53D2702339FF6442932
:10E5F80003D39FF64F2808119EF55E2807D19EF594
:10E608006C2D04119EF4752F01D09EF47C2D0433DB
:10E618009EF3822B04D09EF3872E05119EF28B3534
:10E6280007D09EF2903D01119FF1954203D09FF0D3
:10E6380094400333A0F09F3F0BD0A0F0A13D0F37CB
:10E64800A0EFA33C0DD1A1EFA43C0C33A1EFA43C57
:10E658000AD0A1EEA53D0533A2EEA63C00D1A2EE5C
:10E66800A8390211A3EEAA3C04D0A3EEAD3F0511D0
:10E67800A4EEB24008D0A4EE03410C11A5EE064169
:10E688000AD2A5EE08450711A6EF094A05D2A6EF5A
:10E69800094C0111A7EF0A4807D3A7F00B420B1149
:10E6A800A8F00B420DD4A8F00D461311A9F111469C
:10E6B80014D9A9F1173F1B11A9F21E381ADAA9F3C8
:10E6C80021381811A9F31F3A17DFA9F418391511C1
:10E6D800AAF4163A1DDCAAF5183C1A11AAF51C3A38
:10E6E8001AD9AAF61F391A11ABF6203615D9ABF785
:10E6F80021341711ABF8203B19D9ABF81E3F17117D
:10E70800ACF91D4011D9ACF91E3F0E11ACFA1F40EF
:10E718000CD6ACFB22410D11ACFC23450FD6ADFC49
:10E7280023490B11ADFD214A0DD6ADFE2047091135
:10E73800ADFE21450CD6ADFF22430E11AE00224599
:10E748000CD8AE01214B0A11AE0220500DD7AF03F1
:10E758001D4F0B11AF031A5109D9AF04174A0D11F8
:10E76800B00418470BDBB0051A500A11B0061C5547
:10E778000ED7B1071C560B11B10719470ED9B108AE
:10E78800173C0C11B208183D0CDCB2091C490E11DB
:0DE79800B20A1E4E0AD9B30B1D500B11B36F
:10E7A5000C1A5109D9B30C174F0711B40D17490BA2
:10E7B500DBB40D17480D11B50E19490ADCB50F1953
:10E7C5004F0B11B50F185605DBB61017550711B6C7
:10E7D50011174C0ADBB61116430B11B711173F0D74
:10E7E500DDB71219430C11B7131A480BDCB8131A0D
:10E7F500450F11B81419410DDCB81418400B11B9A7
:10E805001518430DDBB91618470F11B91618490D20
:10E81500DBBA1718470A11BA1717450CDBBB1814D2
:10E82500460F11BB18134C0EDBBC1912510A11BC53
:10E835001A125007DBBC1A12470B11BD1A10400DF6
:10E84500DCBD1B10400A11BE1B124509DCBE1C15A0
:10E85500490B11BE1D184A0ADBBF1D1B4A0811BF13
:10E865001E1B480CDBBF1F1A470E11BF1F1A490B91
:10E87500DBC0201B4B0D11C0211C4910DBC0211D25
:10E88500470F11C1221D4711DBC1231C4B0F11C1BD
:10E89500231B4B0EDBC22419441111C224193D0F51
:10E8A500DBC2251B3B1011C2261D3F0DDAC2261EF9
:10E8B500411011C3271D3F12DAC3271C3D0F11C399
:10E8C500281B3D10DBC4291C401111C4291C450F10
:10E8D500DCC42A1C460E11C42A1B4510DCC52B19A5
:10E8E500431111C52C184511DDC62C164A1011C649
:10E8F5002D174A11DEC62D18491211C72E194710BA
:10E90500DEC72F1A460E11C72F1C4410DFC7301F54
:10E91500471111C731214B0CDBC832224D0E11C8EE
:10E9250032224A10DAC83321471111C83420460F64
:10E93500D9C83520461111C93521430CDBC9362309
:10E945003F0F11C937253D11DBC93725400E11C9C8
:10E9550038254211DCC93925431311C9392543121C
:10E96500DCC93A25431111CA3B24400DDCCA3C24BD
:10E97500411011CA3C23400EDCCA3D22401111CA88
:10E985003E20420FDECB3E20451011CB3F204714E1
:10E99500DECB4021441211CB40213F10DFCB412279
:10E9A5003C0D11CB42234011DFCC42233E1111CC4B
:10E9B50043202F0EE0CC4319221211CC4312201113
:10E9C500E3CC4311250E11CD43132B10E3CD441297
:10E9D5002D1111CD440F2B0FE3CD44092B1211CE70
:10E9E5004404320FE2CE4401360E11CF44B3370D45
:10E9F500E0CF44B3330E11D04401370EE0D04405C7
:10EA05003D0D11D0450A3B0CE3D14512330D11D113
:10EA1500451A2D0EE3D1461E2B0F11D1461D2E0F83
:10EA2500E4D1471D300F11D1471E320EE3D24821E4
:10EA3500330F11D248233510E2D24923350F11D2B5
:10EA45004A20360EE3D24A1D360E11D24B1B341026
:10EA5500E3D34B1B320F11D34B1B300EE4D34C1BAE
:10EA6500340D11D34C1B3A0DE5D44D1A3B0E11D480
:10EA75004D1B360AE6D44E1D340E11D44E1E360DEE
:10EA8500E5D44F1F360C11D5501F350EE5D5501F57
:10EA9500340D11D5511E340EE5D5511E370C11D547
:10EAA500521E390EE5D652203B0F11D653223C0F8C
:10EAB500E4D65423391111D654243710E3D65524FE
:10EAC500360F11D655253310E3D65626330D11D6FC
:10EAD5005627350BE2D657273A0C11D658273C0F47
:10EAE500E2D75827391011D75927370FE2D75A27B8
:10EAF500381011D75A283B0FE2D75B293C1111D7A3
:10EB05005C2B3C12E2D75C2D391111D75D2C3910E5
:0DEB1500E3D75E2B3C0F11D75E293B0EE3CA
:10EB2200D75F27371011D75F26360EE3D760273C11
:10EB32000E11D761284310E3D76229451111D7621C
:10EB4200293F0FE4D763283A1011D763293A11E419
:10EB5200D7642A3E1011D7652C4211E4D7662E42A3
:10EB62001011D7662D3F11E4D7672F3A1011D768DD
:10EB72002D3B0CE4D7682E3D0711D7692E4204E4E1
:10EB8200D76A2E470111D76B2E4702E4D76B2D406F
:10EB92000513D76C2B3503E4D76C2A2B0711D76DDD
:10EBA2002B2909E5D76D2B300611D76E2A3A04E4DA
:10EBB200D76F28400611D76F283E08E4D770273850
:10EBC2000C11D87026320DE6D871252F0911D87193
:10EBD20024310AE9D87221340811D8721B3A08EAA2
:10EBE200D9730D420A11D973104909EADA730C4537
:10EBF2000811DA730A3B06E8DB74093D0211DB7483
:10EC02000A4003E9DB740B3C0213DC75103406EA9C
:10EC1200DC7517350333DC761A3F06EADD771C46CE
:10EC22000433DD771F4001E8DD7824360731DD78D3
:10EC32002C3206E7DC7933320413DC79373409E706
:10EC4200DC7A3A340C33DC7A3C3508E7DC7B3D373E
:10EC52000233DB7C3C3A05E7DB7C3C3D0333DB7D66
:10EC62003B3A04E7DB7D3B320331DA7D3E2D09EA94
:10EC7200DA7E43270D11DA7E4D230AE9DA7E572622
:10EC82000B11D97D5E2C0BE9D97D61300C11D97D38
:10EC9200632F08EAD87D662F0511D87C683005EA13
:10ECA200D87C6D330611D77B733608E9D77B7C3865
:10ECB2000511D77A853A04E8D8798B3B0711D879C0
:10ECC2008E3809E9D8788F371011D878903B0BE845
:10ECD200D87791420D11D976954A08E7D9769849A5
:10ECE2000411D9759D4008E8DA75A23A0B33DA753A
:10ECF200A53C0AE8DB75A8430031DB74AA4603E9A8
:10ED0200DC74AF460213DC74004A02EADD75054C7E
:10ED12000333DD75084D00EDDE75084B0533DF76F4
:10ED2200064902EDDF76044A0131E076044902EA3F
:10ED3200E076044C0513E176045006EAE176014DD3
:10ED42000D33E276B1450FEAE276AD3F1077E37517
:10ED5200AB3F0DEAE375AC430A33E475AE4604EA11
:10ED6200E475B0400131E575B23908EAE575013C58
:10ED72000611E675054607ECE6760A4B0311E776BF
:10ED82000F4604EEE777163B0611E778203405ECD0
:10ED9200E77827350611E7792D3409ECE779323423
:10EDA2000B11E77A3B260AECE67A45250B11E67A47
:10EDB2004D230BEAE67A56250711E67A5F270AEA1F
:10EDC200E579672A0C11E579731F0AEBE578792E4C
:10EDD2000811E578843302EAE5778D3B0313E67682
:10EDE200954104EAE676993F0733E6759A3801EAD7
:10EDF200E67595310531E6748F3202EAE6748E3596
:10EE02000111E773923301EAE77398310413E77251
:10EE12009D3304EBE872A1370911E872A33F0DEBB1
:10EE2200E971A5471091E971A94D0CEBEA71AA4865
:10EE32000D11EA71AD480CECEB71AE4C0E11EB709A
:10EE4200AE5012ECEC70AF501711EC70AF4A1AECE6
:10EE5200ED70B2481711EE70004D15ECEE700250D5
:10EE62001811EF70024A11EEEF7002410D11F071AC
:10EE7200023F0DEDF07102470F11F171034F0CEDDE
:10EE8200F171054D0E11F271084812EFF272094547
:0DEE92001511F372094514EFF3720A4712CF
:10EE9F0011F4720B4914EFF4730F461111F473133D
:10EEAF003F14F0F57418381811F5751E3716EFF575
:10EEBF0075233B1411F576273C16EDF5772A39119A
:10EECF0011F5772B3811EDF5782B381311F5782ACA
:10EEDF003918EEF5792A3C1A11F57A2C3C20EEF50B
:10EEEF007B2E3D1C11F57B2F4028EEF57C2F4230F9
:10EEFF0011F57D2D4114EFF57D2D3D3811F57E2C4B
:10EF0F00393AF0F57F2B3B3C11F57F2B403CEFF569
:10EF1F00802C453A11F5812C4639EFF5822C433B75
:10EF2F0011F5822A3F3DEFF583293D3C11F5842AE7
:10EF3F003D3BF0F5852B413611F5852A4434F1F52B
:10EF4F00862A423211F587293F2EF2F5872A3D286E
:10EF5F0011F5882B3C22F2F5892C401E11F58A2ED3
:10EF6F00451BF2F58A2D451611F58B2D4113F2F540
:10EF7F008C2C3C1111F58C2E3812F2F58D30391581
:10EF8F0011F58E2F3B13F2F58E2D3A1211F58F2CB2
:10EF9F003715F3F58F2C331911F5902F3117F3F532
:10EFAF009132341711F591343C13F3F592343D112E
:10EFBF0011F593333A0EF3F59332390D11F494336F
:10EFCF003C0FF4F49534411111F495344416F3F4D5
:10EFDF009635411811F497363C14F3F497363911DE
:10EFEF0011F498353C13F4F399343F1411F3993419
